:0200000480007A
:10000000B72F0000938F0F8073900F3015A8130047
:100010000000130000001300000013000000130094
:100020000000130000001300000013000000130084
:100030000000130000001300000013000000010086
:10004000970200009382020C73905230814001416C
:100050008141014281420143814301448144014580
:100060008145014681460147814701488148014950
:100070008149014A814A014B814B014C814C014D20
:10008000814D014E814E014F814F971102009381A6
:10009000A1DA170502001305E55E97A50300938515
:1000A00025880146112217050200130565529705A0
:1000B0000200938525580146C52817B5030013058E
:1000C000658697C503009385A58537B6ABAB130648
:1000D000B6BAD92817C103001301C184EF70B03438
:1000E000860293D21200F512638802008242110147
:1000F0006F00001073002030824211017300203025
:10010000711116C0F3222034E3CC02FC82421101AB
:10011000130141F806C20AC40EC612C816CA1ACC88
:100120001ECE22D026D22AD42ED632D836DA3ADCC7
:100130003EDEC2C0C6C2CAC4CEC6D2C8D6CADACC97
:10014000DECEE2D0E6D2EAD4EED6F2D8F6DAFADCA7
:10015000FEDE73252034F32510340A8601A07310C7
:10016000153492402241B2414242D2426243F243AC
:10017000025492542255B2554256D2566257F25703
:10018000064896482649B649464AD64A664BF64B33
:10019000065C965C265DB65D465ED65E665FF65F83
:1001A0001301C1077300203010C16374B50011053D
:1001B000E5BF828000000000000000000000000099
:1001C000000000000000000000000000000000002F
:1001D000000000000000000000000000000000001F
:1001E000000000000000000000000000000000000F
:1001F000197106C00AC20EC412C616C81ACA1ECC8D
:1002000022CE26D02AD22ED432D636D83ADA3EDCC6
:1002100042DEC6C0CAC2CEC4D2C6D6C8DACADECC96
:10022000E2CEE6D0EAD2EED4F2D6F6D8FADAFEDCA6
:100230009702020083A2023D23A02200F322103481
:1002400096DEEF00002B170102000321A13B0241C3
:10025000F65273901234B72200009382028873A082
:10026000023082403242C2425243E24372448254DC
:100270001255A2553256C2565257E2577258864806
:100280001649A649364AC64A564BE64B764C865C1A
:10029000165DA65D365EC65E565FE65F0961730059
:1002A0002030970202009382E23D23A0120023A295
:1002B000220023A4320023A6420023A8520023AA2E
:1002C000620023AC720023AE820023A0920223A21C
:1002D000A20223A4B20223A6C20223A8D20223AA06
:1002E000E20223ACF20223AE020323A0120523A2F2
:1002F000220523A4320523A6420523A8520523AADA
:10030000620523AC720523AE820523A0920723A2C7
:10031000A20723A4B20723A6C20723A8D20723AAB1
:10032000E20723ACF207EF40702717010200032118
:10033000612D0241F65273901234B722000093826D
:10034000028873A0023082403242C2425243E243EA
:10035000724482541255A2553256C2565257E25731
:10036000725886481649A649364AC64A564BE64B45
:10037000764C865C165DA65D365EC65E565FE65FB1
:10038000096173002030970202009382A22F83A09C
:10039000020003A1420083A1820003A2C20083A243
:1003A000020103A3420183A3820103A4C20183A427
:1003B000020203A5420283A5820203A6C20283A60B
:1003C000020303A7420383A7820303A8C20383A8EF
:1003D000020403A9420483A9820403AAC20483AAD3
:1003E000020503AB420583AB820503ACC20583ACB7
:1003F000020603AD420683AD820603AEC20683AE9B
:10040000020703AFC20983AF820782807370043092
:10041000197106C00AC20EC412C616C81ACA1ECC6A
:1004200022CE26D02AD22ED432D636D83ADA3EDCA4
:1004300042DEC6C0CAC2CEC4D2C6D6C8DACADECC74
:10044000E2CEE6D0EAD2EED4F2D6F6D8FADAFEDC84
:100450009702020083A2021B23A0220086DEEF2067
:10046000602E170102000321E1190241F652739038
:100470001234B72200009382028873A002308240B7
:100480003242C2425243E243724482541255A25550
:100490003256C2565257E257725886481649A649F4
:1004A000364AC64A564BE64B764C865C165DA65DD0
:1004B000365EC65E565FE65F09617300203073707A
:1004C000043001A07310453082807325403073F0F2
:1004D00043308280970700009387A7FE232EB5FE46
:1004E0002322C5FA232635F82320F5F8130505F84D
:1004F0008280411106C6EF409007EF10900A01E597
:10050000B24041018280B24041016F20A023930795
:1005100085007D575CC118C55CC51CC9232005003A
:1005200082802328050082805C41DCC1984798C501
:1005300098474CC38CC788C91C4185071CC1828061
:100540009041FD57130785006314F60039A83E87D4
:100550005C439443E37DD6FEDCC18CC798C54CC395
:1005600088C91C4185071CC1828018495C43EDB7CE
:10057000584114451C4914C71845544154C3D84325
:100580006314A7001845D8C32328050088437D15A8
:1005900088C382803041AE8701CE4C455841B29528
:1005A0004CC563E4E5000C414CC53E856F30B0207E
:1005B0008280411122C406C62A8426C2EF2030124E
:1005C0003C44635BF0025C5085CB9304440209A871
:1005D0003C44FD173CC43C446350F0025C5089CF5E
:1005E0002685EF2040586DD5EF2020783C44FD173C
:1005F0003CC43C44E344F0FEFD573CC4EF20701083
:10060000EF20F00D7C40635BF0021C4885CB930427
:10061000040109A87C40FD177CC07C406350F002B7
:100620001C4889CF2685EF2000546DD5EF20E0735C
:100630007C40FD177CC07C40E344F0FEFD577CC04D
:100640002244B240924441016F20B00B29CD0111E8
:1006500022CC2A8406CE26CA4AC84EC62E89EF204E
:10066000100824404C5C832904002685EF708038F4
:100670007D57232C0402B3079540CE974E9578C042
:1006800048C0232434015CC438C4631109021C48E7
:100690008DE7EF201007F2406244D2444249B2494C
:1006A0000545056182807370043001A013050401C3
:1006B000B93D13054402A13DE9BF13050401EF2034
:1006C000804A8547E317F5FC9133E1B701E5737084
:1006D000043001A0011126CA4AC84EC606CE22CC5B
:1006E000AA842E89B289A5C9EF70C03013055505BB
:1006F000EF3020742A8435C5930745051CC144DCBE
:1007000023202405EF20A07D24404C5C0329040015
:100710002685EF70202EFD56232C0402B30795404A
:100720003307A900CA9774C058C05CC434C4130509
:10073000040123242401E13B13054402C93BEF20BB
:10074000407C230834052285F2406244D244424969
:10075000B2490561828013054005EF30806D2A841F
:1007600001E57370043001A000C051BF01E5737052
:10077000043001A06375B5007370043001A041110D
:1007800022C409462E84814506C6893711C500DD7D
:10079000B2402244410182807370043001A05D7137
:1007A00086C6A2C4A6C2CAC04EDE52DC56DA5AD8E9
:1007B0005ED632C6630A051C6382051C89476399AD
:1007C000F600585D85476305F7007370043001A09B
:1007D0003689AE842A84EF20C05B11E5B24781C719
:1007E0007370043001A0EF20806F185C5C5C014BDB
:1007F000894BFD59130A0401930A44026365F70CFF
:1008000063077919B2476381072463150B00280831
:10081000EF208048EF20E06EEF10604FEF20206C5B
:100820007C4063943701232204043C4463943701E1
:1008300023240404EF20E06C6C002808EF20E0473C
:10084000631E051EEF20A069185C5C5C630CF70A50
:10085000EF20206BEF20A0683C44634FF00039A8E4
:100860005685EF20403019C1EF2020503C44FD1741
:100870003CC43C446354F0005C50FDF32324340535
:10088000EF202068EF20A0657C40634FF00039A87E
:100890005285EF20402D19C1EF20204D7C40FD17DF
:1008A0007CC07C406354F0001C48FDF323223405D7
:1008B000EF202065EF10A06A054BEF204062185C26
:1008C0005C5CE37FF7F230406305060C631F09129E
:1008D0000844A685EF30206E1C4434405840B6973B
:1008E0001CC463EAE70A1C5C14405850850714C412
:1008F0001CDC5DC713054402EF20E0268547631129
:10090000F50AC9A8EF20E05FB2455285EF206007E5
:10091000EF20E05C3C44634FF00039A85685EF209F
:10092000802419C1EF2060443C44FD173CC43C4482
:100930006354F0005C50FDF323243405EF20605C29
:10094000EF20E0597C40634FF00039A85285EF203A
:10095000802119C1EF2060417C40FD177CC07C40A4
:100960006354F0001C48FDF323223405EF20605946
:10097000EF10E05E31F1593C054B81B73C41E38F0C
:1009800007E27370043001A07370043001A030409E
:1009900021E61C4085C71C5C585085071CDC39FBD0
:1009A000EF2020560545B640264496440649F259A4
:1009B000625AD25A425BB25B616182804840EF204A
:1009C00060491C5C58502322040085071CDCE3139B
:1009D00007F279D5253CE9B74844A685EF30A05DFC
:1009E0003C4058441440B307F0403E9758C4637CE1
:1009F000D7025840BA975CC409475C506306E902C5
:100A0000185C050718DCC9DFF5B54844A685EF304A
:100A1000805A3C4058441440B307F0403E9758C4B5
:100A2000E37CD7FCF9B75C50185C79DB185C7D1768
:100A300018DC185C050718DCA5D76DBD2285953E2E
:100A4000EF10E051014585B7EF20A04B0145A1BF54
:100A5000411126C2AA841305400522C406C6EF3000
:100A6000403D2A8415CD232C0502FD577CC1054746
:100A7000410558DC3CC42322040023200400232425
:100A80000400232604002320040423089404413492
:100A900013054402AD3C8146014681452285013360
:100AA0002285B24022449244410182800DC5411109
:100AB00022C426C206C64AC0032945002A84EF2064
:100AC000802C8144630CA900B2402244268502494F
:100AD0009244410182807370043001A05C448544DB
:100AE000FD175CC4F5F381460146814522854539F1
:100AF000E1BF31CDA1C9011122CC26CA4AC852C4D6
:100B000006CE4EC68947B68432892E8A2A846399D6
:100B1000F600585D8547630FF7047370043001A039
:100B20006D32185C5C5CAA896366F70281444E856D
:100B3000513AF240624426854249D244B249224A9F
:100B4000056182803C41C5DB7370043001A0737085
:100B5000043001A0304041E21C40D5CB1C5C7D57E5
:100B600085071CDC3C446387E7083C4485448507D3
:100B70003CC475BF993A185C5C5CAA89636DF70246
:100B8000304079DA4844D285EF30E0423C40584466
:100B90001440B307F0403E9758C46375D7005840DF
:100BA000BA975CC48947E39BF4FA1C5CC5DB1C5C08
:100BB000FD171CDC65B7304045D24844D285EF3084
:100BC000803F3C4058441440B307F0403E9758C41F
:100BD000E367D7FCD9BFDDF40844D285EF30A03DF0
:100BE0001C4434405840B6971CC4E3E9E7F61C4067
:100BF0001CC4ADB75C5085449DDB13054402EF1067
:100C0000907615D5E30509F2232099000DB74840E9
:100C1000EF2040242322040091B721CD3C4181C71D
:100C20007370043001A01C41A1CB011122CC26CA53
:100C30002A844AC84EC606CE2E894138185C5C5CB0
:100C4000AA898144637DF7001C5C7D5785071CDC05
:100C50003C446388E7023C44854485073CC44E8598
:100C60009530F240624426854249D244B24905613A
:100C700082807370043001A05C41C5DB7370043066
:100C800001A05C5099E38544D9BF13054402EF10DD
:100C9000906D75D9E30909FE85472320F900E5B772
:100CA000397106DE22DC26DA4AD84ED652D456D224
:100CB00032C66302051C638A051AB68AAE892A8485
:100CC000EF20200D11E5B24781C77370043001A0F9
:100CD000EF20E0201C5C63920714B247638E070A82
:100CE0002808EF10707BFD5413094402130A040115
:100CF000EF202021EF10A001EF20601E7C406394C4
:100D00009700232204043C446394970023240404A2
:100D1000EF20201F6C002808EF10307A63130518AD
:100D2000EF20E01B1C5CADCFEF20A01DEF20201BAF
:100D30003C44634FF00039A84A85EF10D06219C1D6
:100D4000EF20A0023C44FD173CC43C446354F00037
:100D50005C50FDF324C4EF20C01AEF2040187C4003
:100D6000634FF00039A85285EF10F05F19C1EF1002
:100D7000D07F7C40FD177CC07C406354F0001C4851
:100D8000FDF364C0EF20E017EF10601DEF20201589
:100D90001C5CC1E7B247A9FFEF20A016014555A092
:100DA000EF2020161C40DDC7B2454A85EF10703D8C
:100DB000EF20E0123C44634FF00039A84A85EF1061
:100DC000905A19C1EF10707A3C44FD173CC43C4462
:100DD0006354F0005C50FDF324C4EF208012EF2038
:100DE00000107C40634FF00039A85285EF10B057D7
:100DF00019C1EF1090777C40FD177CC07C40635494
:100E0000F0001C48FDF364C0EF20A00FEF10201588
:100E100031C9EF20C00C1C5CB5DFCE85228544446F
:100E2000EFF04FF7639C0A041C5C1840FD171CDCB4
:100E300001E7EF20801148C01C48A1EFEF20600CB3
:100E40000545F2506254D2544259B259225A925A2C
:100E500021618280EF20A0084840EF109075EF20BC
:100E6000400A99B7EFF08FDA6DB73C41E38707E4AA
:100E70007370043001A07370043001A05C5044C44E
:100E8000D5DF13054402EF10104E4DD9EFF00FD807
:100E900075B713050401EF10104D8547E310F5FAFF
:100EA000F5B72285EFF0EFF0EF10600B014551BF71
:100EB0001DC9411122C44AC006C626C244412E891A
:100EC0002A84EF10506C6383A40281464A868145D0
:100ED0002285F93385476300F502B24022449244EB
:100EE0000249410182807370043001A05C440545D1
:100EF00085075CC4DDB75C4485075CC4F9BF15CDCC
:100F0000ADC9011122CC26CA4AC84EC652C42A8491
:100F100006CE3289AE89EFF04FDB1C5C2A8A814411
:100F200085E35285EFF00FDAF240624426854249AC
:100F3000D244B249224A056182807370043001A014
:100F4000304001CE4C445C40B2954CC463E4F500A3
:100F50000C404CC44E85EF3000061C5C7D57FD17DD
:100F60001CDC7C40638CE7007C40854485077CC0AA
:100F70004DBF3C41D9D77370043001A01C4899E3A0
:100F8000854445B713050401EF10F03D75D9E30919
:100F900009FE85472320F900E5B721C93C41A1CDD1
:100FA000A1CB011122CC26CA4AC852C42A8406CE3B
:100FB0004EC62E8AEFF06FD11C5C2A89814491CBFA
:100FC0008329C400D2852285EFF0CFDC8544232617
:100FD00034014A85EFF00FCFF24062442685424942
:100FE000D244B249224A056182807370043001A064
:100FF0007370043001A0EDDF7370043001A001E5CF
:101000007370043001A0411122C42A8406C6EF1077
:10101000106D005CEF10F06EB24022852244410159
:10102000828001E57370043001A0411106C622C41C
:101030002A84EF10D06A1C5C405C1D8CEF10706C31
:101040002285B24022444101828019C1085D82801C
:101050007370043001A01DCD979703009387878894
:10106000D843630CE502D847630CE504D84B63070B
:10107000E504D84F6302E504D853630DE502D85761
:101080006308E502D85B6303E502D85F630EE50001
:101090006F20506C7370043001A001470E07BA979F
:1010A00023A007006F20106B1D47CDBF1947FDB768
:1010B0001547EDB71147DDB70D47CDB70947F9BF64
:1010C0000547E9BF684582806CC5828003450505F8
:1010D000828009C5085D1335150082807370043065
:1010E00001A019C51C5D485D1D8D1335150082805A
:1010F0007370043001A0978703009387A77E9843FD
:1011000005C3984705C7984B05C7984F05C798531F
:1011100005C7985705C7985B15C7985F15C38280A8
:1011200001470E07BA978CC3C8C382800547D5BF55
:101130000947C5BF0D47F5B71147E5B71547D5B7FF
:101140001D47C5B71947F1BF978703009387877974
:10115000D8436308E502D847630BE502D84B630A1E
:10116000E502D84F6309E502D8536308E502D85772
:101170006307E502D85B6308E502D85F6303A70253
:10118000828001470E07BA9723A007008280054797
:10119000D5BF0947C5BF0D47F5B71147E5B7154797
:1011A000D5B71D47C5B71947F1BF411122C426C2A3
:1011B0004AC02A8406C6AE843289EF105052784065
:1011C000FD576314F700232204043844FD576314C9
:1011D000F70023240404EF10D0521C5C99E74A86E0
:1011E000A68513054402EF10D00CEF10504F3C447D
:1011F000635BF0025C5085CB9304440209A83C4435
:10120000FD173CC43C446350F0025C5089CF2685F6
:10121000EF1070156DD5EF1050353C44FD173CC4F0
:101220003C44E344F0FEFD573CC4EF10904DEF10FA
:10123000104B7C40635BF0021C4885CB9304040197
:1012400009A87C40FD177CC07C406350F0021C481C
:1012500089CF2685EF1030116DD5EF1010317C400D
:10126000FD177CC07C40E344F0FEFD577CC0224467
:10127000B2409244024941016F10B0481DC17971DA
:101280004ECE52CC06D63E8A22D426D24AD056CA58
:101290005AC85EC6A547BA8963F8E7007370043080
:1012A00001A07370043001A02A8BAE843289B68B02
:1012B000C28A6307082213050006EF2090372A84AC
:1012C000630B05200A09232855034A869305500A13
:1012D0005685EF20505C03C704001C587119230A7F
:1012E000E40203C704003E991379C9FF79C783C795
:1012F0001400A30AF40283C71400E1C383C72400C7
:10130000230BF40283C72400CDCB83C73400A30B87
:10131000F40283C73400D5C383C74400230CF4020E
:1013200083C74400D9CB83C75400A30CF40283C7FE
:101330005400C1C783C76400230DF40283C764004F
:10134000ADCF83C77400A30DF40283C77400B5C783
:1013500083C78400230EF40283C78400B9CF83C7F8
:101360009400A30EF40283C79400A1CB83C7A4000A
:10137000230FF40283C7A400A9C383C7B400A30F3B
:10138000F40283C7B40095CB83C7C4002300F404E0
:1013900083C7C4009DC383C7D400A300F40483C7DC
:1013A000D40081CF83C7E4002301F40483C7E400A1
:1013B00089C783C7F400A301F404930A4400568547
:1013C000A30104042326340323283405232A040418
:1013D000EFF02F9513058401EFF0AF94A947B38781
:1013E0003741232C040400C81CCC40D02322040421
:1013F000232E04045E86DA854A85EFF0AF8D08C09F
:1014000063040A0023208A007370043017F9010076
:101410001309891D8327090097F401009384841E12
:1014200091C798409C407C4385077CC317F7010017
:101430001307471C1C43850797F6010023ACF61AD7
:101440009C40C5CB8327090017FB0100130B4B2BD6
:1014500089EB9C40DC5763E6F90097F7010023A372
:10146000871A97F70100938727179C4317F7010006
:101470001307C71748541843850797F6010023AD93
:10148000F6143CC46376A70097F7010023A0A716C3
:10149000D145EF602056D6855A95EFF0EF88832727
:1014A000090081C79C40FC43B5E38327090005443C
:1014B00099C79C40DC5763F43701EFE03FF5228584
:1014C000B250225492540259F249624AD24A424BD3
:1014D000B24B456182805685EF20D0277D54C5B739
:1014E00013152600EF20F014AA8AE31605DC7D54BC
:1014F000F9B797F7010023A78710184385476301C1
:10150000F70217FB0100130BAB1FA1BF98409440DB
:101510007C43FD177CC3FC42C9FB7360043071B788
:10152000014A17FB0100130BAB1DA94B5285D14596
:10153000EF60404C050A5A95EFE07FFDE3187AFF13
:1015400097FB0100938B4B285E85EFE05FFC17FA59
:101550000100130AAA285285EFE07FFB17F501006E
:1015600013050529EFE0BFFA17F5010013058529DA
:10157000EFE0FFF917F501001305052AEFE03FF949
:1015800097F7010023AE770797F7010023A84707D5
:10159000C9BD411122C406C626C24AC02A8473703E
:1015A000043097F40100938424049C40F9E311E48F
:1015B00097F70100938707058043130944004A8584
:1015C000EFE01FFB1C5489C713058401EFE05FFAAD
:1015D000CA8517F501001305E522EFE0FFF497F740
:1015E000010093876701984397F701009387C7FE2F
:1015F0009C43050797F6010023A0E6009840850765
:1016000097F6010023AAF6FC01CB97F70100938718
:1016100067FF9843784349EF9C40B1C797F70100B3
:10162000938747FE9843630F870873700430984090
:1016300039EB17F701001307A7FC14439442A5E206
:101640007D5797F6010023A7E6F8984009CF984305
:10165000784311CB984394437C43FD177CC3FC42F1
:1016600099E373600430B24022449244024941013C
:10167000828097F701009387E7F898439C437C4367
:1016800085077CC32DB794439843F8420507F8C2F9
:1016900017F701001307C7F614439442D5D2184335
:1016A00058475847584397F6010023A5E6F271BF03
:1016B000984394437C43FD177CC3FC42B1FF7360A5
:1016C000043099BF97F70100938787F09C4381C747
:1016D0007370043001A02244B24092440249410197
:1016E0006FE0DFD241C517F701001307A7F11443DC
:1016F0008147638BA606411106C622C426C27370B9
:10170000043097F60100938626EE9C4291C7104361
:101710001C437C4285077CC29C42AA84404981C705
:101720001C43FC43B9E797F70100938767ED9C439F
:10173000638B870497F70100938747EC9C4363848E
:10174000870497F701009387270D6309F40297F741
:1017500001009387270B6301F4028547B2402244BE
:1017600092443E85410182803E85828073700430C0
:1017700001A0EF60A04045BF9147CDB79C5493B7FF
:1017800017008907E1BF8947D1BF7370043097F70D
:101790000100938767E5984309EF15C59C434855B9
:1017A00081CB97F701009387E7E59843784315E3EA
:1017B000828017F701001307E7E414431843F84247
:1017C0000507F8C261FD17F701001307A7E30843F7
:1017D000F1B7984394437C43FD177CC3FC42E9FB7B
:1017E000736004308280411122C42A8406C6EFE06F
:1017F000DFCD11E497F701009387C7E080434054A1
:10180000EFE05FCCB2402285224441018280A547AF
:1018100063F5B7007370043001A0011122CC06CE2D
:1018200026CA4AC84EC652C42A847370043017F9B7
:101830000100130969DB83270900CDEF71C43C481F
:101840006388F50817F701001307C7DB63FCB700CF
:101850001443638C860C18434457B3B4950093C467
:10186000140029A00443818C93B41400585463835A
:10187000E70A1C4C2CC863C60700A947B385B740CC
:101880000CCC93172700BA97584897F90100938911
:1018900029E78A07CE97631AF702130A4400528594
:1018A000EFE01FCD97F70100938747D448549C433E
:1018B00063F6A70097F7010023AAA7D2D145EF60EE
:1018C0006013D2854E95EFE03FC699C0EFE01FB49C
:1018D0008327090081CB97F701009387A7D29C4308
:1018E000FC439DEBF2406244D2444249B249224A51
:1018F0000561828097F701009387C7D098439C4386
:101900007C4385077CC305FC97F70100938787CF4D
:10191000804335B74CD4B1BF6244F240D24442490F
:10192000B249224A05616F606025814481B725C1B3
:10193000011126CA97F401009384C4CC9C4006CEC2
:1019400022CC4AC84EC6638DA7027370043017F9C3
:101950000100130969C98327090091C798409C4079
:101960007C4385077CC3584997F701009387C7EAF2
:101970006302F7028327090081C79C40FC43A5EB63
:10198000F2406244D2444249B24905618280737098
:10199000043001A01C5517F70100130767E5E38B1E
:1019A000E7FCE9FB930945002A844E85EFE05FBC24
:1019B00097F70100938787C348549C4363F6A700B9
:1019C00097F7010023A4A7C2D145EF60A00297F7C3
:1019D00001009387E7D23E95CE85EFE0FFB49C40AF
:1019E0005854DC57E368F7F8EFE05FA261B7624450
:1019F000F240D2444249B24905616F60201815CDCA
:101A0000011122CC26CA4EC62A8406CE4AC8EFE06F
:101A1000DFAB584897F70100938707E0AA89814414
:101A20006300F7024E85EFE0FFA9F240624426858D
:101A30004249D244B249056182807370043001A0EA
:101A40001C5417F501001305A5DAE38DA7FCF9FB7B
:101A500097F701009387C7B79C43A9EB97F701005D
:101A6000938747BA9C43445413094400DC574A8582
:101A7000B3B4F400EFE0DFAF97F70100938707B747
:101A800048549C4393C4140063F6A70097F70100E1
:101A900023AEA7B4D145EF50F07597F701009387B7
:101AA00027C6CA853E95EFE03FA8ADBF93058401E8
:101AB000EFE09FA785BF0111056506CE22CC26CA9F
:101AC0004AC84EC652C456C25AC0EF208036630E72
:101AD000051AAA8413050006EF20A0352A84630A9C
:101AE000051C05669305500A04D92685EF20A05AE7
:101AF00004588567F117BE94B7474C4593879744C0
:101B0000130A44005CD85285230C0402A301040488
:101B10002326040223280404232A0404EFE07FA0E0
:101B200013058401EFE0FF9FA947232C0404F198DB
:101B300000C81CCC40D023220404232E04040146F8
:101B4000971500009385E5B12685EFE0BF9808C0A2
:101B50007370043017F90100130909A983270900DC
:101B600097F40100938404AA91C798409C407C4359
:101B700085077CC317F701001307C7A71C43850718
:101B800097F6010023A8F6A69C40C9C38327090045
:101B900097F901009389C9B681EB9C40DC5789E72E
:101BA00097F7010023A087A697F701009387C7A2A4
:101BB000984397F60100938666A35C549442050708
:101BC00017F60100232AE6A038C463F6F60017F7DB
:101BD0000100232DF7A0139527003E950A05D28515
:101BE0004E95EFE07F948327090081C79C40FC431A
:101BF000DDE78327090091C39C40EF10F04985473A
:101C00006305F50C59E17370043001A097F70100EA
:101C100023AA879E1843854797F90100938949AE07
:101C2000E314F7F8CE8A17FB0100130BEBB95685C6
:101C3000D10AEFE0DF8DE31C5BFF17F50100130510
:101C4000A5B8EFE0DF8C97FA0100938A2AB9568590
:101C5000EFE0FF8B17F50100130585B9EFE03F8B2F
:101C600017F50100130505BAEFE07F8A17F50100AB
:101C7000130585BAEFE0BF8997F7010023A26799A2
:101C800097F7010023AC579705B7F2406244D2445E
:101C90004249B249224A924A024B056182809840E9
:101CA00094407C43FD177CC3FC42A1F77360043071
:101CB00089B76244F2404249B249224A924A024BF1
:101CC0002685D24405616F20E02873700430FD57EB
:101CD00017F701002320F790624497F7010023A52E
:101CE000A790F240D2444249B249224A924A024B5A
:101CF00097F7010023AE078E05616FE08FDA7370EE
:101D0000043097F7010023A1078E6FE0CFE717F7A4
:101D100001001307E78B1C4385071CC38280737087
:101D2000043097F701009387278C984305E317F752
:101D300001001307E78B08439C4381CB97F7010011
:101D40009387478C9843784301EF828017F701000F
:101D50001307478B14431843F8420507F8C2C1BF65
:101D6000984394437C43FD177CC3FC42F9FF7360A6
:101D700004308280411106C622C4EFE00FF597F7C8
:101D800001009387E7868043EFE0CFF3B2402285DE
:101D900022444101828097F701009387A7858843F9
:101DA0008280797106D622D426D24AD04ECE52CC29
:101DB00056CA5AC85EC697F70100938767819C434D
:101DC000B1EF17F701001307A7821C43850797F6A9
:101DD000010023AFF680832A0700638F0A0697E786
:101DE00001009387277F9C43814463F1FA0897F9A8
:101DF00001009389E99017FA0100130AAA8083274A
:101E00000A008546D85793172700BA978A07BE99C4
:101E100083A7090063FFF600854421A897E7010026
:101E20009387477C9C438144850717E70100232B58
:101E3000F77A97E701009387A77A9C4391C385447B
:101E4000B2502254268502599254F249624AD24A2B
:101E5000424BB24B4561828017E401001304447A7F
:101E60001C409C43DDC37370043001A017E40100E3
:101E70001304047997F901009389898817EA01000E
:101E8000130A4A7817EB0100130B4B761C409C4356
:101E9000B5C31C40DC4703A9C70083274900930B47
:101EA00049005E8563EEFA04EFE08FEC8327890238
:101EB0001305890199C3EFE0AFEB8327C90203271C
:101EC0000B00DE85139527003E950A054E95637637
:101ED000F70017E70100232BF770EFE0EFE483270B
:101EE0000A000327C902DC57E362F7FA1C40854465
:101EF0009C43C5F3FD5717E70100232DF76C01B78D
:101F000017E701002328F76CDDBD17E70100130771
:101F1000E76E1C40184397E6010023A3E66E17E71F
:101F20000100232DF76C97E701009387276B9C43F3
:101F3000850717E701002323F76A1C409C4399E7B4
:101F4000FD5717E701002327F76851BD1C40DC4708
:101F5000DC47DC4317E70100232EF76649B597E716
:101F600001009387E766984301E77370043001A08E
:101F7000011106CE22CC26CA4AC84EC652C456C249
:101F80005AC07370043097E401009384E46598406C
:101F900061EB98437D1797E6010023ABE6629C4313
:101FA000D9EB97E701009387E7649C43C9C797EA99
:101FB0000100938AEA7417EA0100130A2A6317E9F9
:101FC000010013092964854919A83385EA00EFE067
:101FD000AFD5832709005854DC576379F70483A7EA
:101FE0000A0FC1CF83A7CA0FC04713058401EFE0D2
:101FF0002FD8130B44005A85EFE08FD75C5483260B
:102000000A00DA85139527003E950A052A8756951A
:10201000E3FDF6FA17E70100232AF75CEFE0CFD0E3
:10202000832709005854DC57E36BF7FA97E7010060
:1020300023A8375B6DB701449C4081CB97E7010033
:102040009387475C9C43FC4395E72285F2406244BA
:10205000D2444249B249224A924A024B05618280E7
:1020600017E701001307075A14431843F8420507FE
:10207000F8C205B7EF509030C9BF17E40100130450
:1020800064561C4095C31C40054999CF193B09C5AE
:1020900097E7010023A627551C40FD1717E701000D
:1020A0002322F7541C40FDF397E701009387475321
:1020B00098438547E311F7F8EFE04FB50544ADBF0E
:1020C00011CD81E57370043001A017E701001307FB
:1020D00027501C4399C77370043001A073700430FB
:1020E00001A0411122C406C614431841850617E613
:1020F0000100232FD64C97E601009386664F944249
:102100003304B70000C163F7E602637FE40063FDB8
:10211000860097E701009387E74E88431105EFE0BB
:102120002FC52285EF50501F1D3D01C9B2402244EA
:1021300041018280E36FE4FCD9BF2244B2404101F7
:102140006FE0CFAC11C917E70100130767481C43C4
:1021500091C77370043001A06FE04FAB411106C608
:1021600022C41843AA87050797E6010023A2E64682
:1021700097E601009386064917E7010013074747D2
:10218000184388423304F7001105EFE06FBE228543
:10219000EF509018E93311E52244B24041016FE05D
:1021A000EFA6B240224441018280411122C406C6FA
:1021B00097E701009387C7419C430144850717E7D0
:1021C00001002327F74097E701009387A7429C432C
:1021D00063E0F51217EE0100130E4E5E97E2010068
:1021E0009382425101440147854F1303500A21A0B5
:1021F000311E638DC20B83278EFFBA86F5DB8327E2
:10220000CEFFDC43232EFEFE638AC70F03AFC70059
:10221000DC432A97814E232EFEFE6385C70783A8E1
:10222000C70093874803232017015CC383A7880452
:102230002326F7011CC783A7C8021CCB83A7080568
:10224000232C07005CCB03A8080383470800639096
:102250006704C287850783C60700B3850741E38B00
:1022600066FE8981C205C181231EB700850E130752
:10227000070263061F038327CEFFDC43232EFEFEE7
:10228000E39FC7F983274E00232EFEFE49BF8145F9
:10229000231EB700850E13070702E31E1FFD769469
:1022A00013175400311EBA86E397C2F597E7010071
:1022B0009387073503AE070083270E00639D070E43
:1022C00097E701009387873303AE070083270E004B
:1022D0006392071817EE0100130E8E4283274E10EB
:1022E0009DE383278E116395072019C223200600E2
:1022F000BD312285B24022444101828083274E00B5
:10230000232EFEFE21B783278E1017EF0100130F37
:10231000EF4FDC4317E701002328F74E6380E733D4
:1023200083A2C700DC43AA96814E17E70100232D44
:10233000F74C914F1303500A6388E70783A8C7003F
:102340009387480323A01601DCC283A7880423A631
:10235000F6019CC683A7C8029CCA83A7080523ACC4
:102360000600DCCA03A80803834708006391672AB4
:10237000C287850703C70700B3850741E30B67FEE4
:1023800093D72500C207C183239EF600850E93864E
:1023900006026386122983278E10DC4317E70100AB
:1023A0002324F746E39CE7F983270E1117E7010082
:1023B000232CF74461B783274E00130F8E00D443BC
:1023C0002322DE006388E629B307E500D84283A212
:1023D000C600814E2322EE00894F1303500A630684
:1023E000EF068328C7001387480323A01701D8C32B
:1023F00003A7880423A6F70198C703A7C80298CBB0
:1024000003A7080523AC0700D8CB03A8080303479C
:1024100008006318671C4287050783460700B30559
:102420000741E38B66FE13D7250042074183239EB5
:10243000E700850E93870702638D121B83264E00EB
:10244000D8422322EE00E31EEFF80327CE0023221A
:10245000EE0041BF83274E00130F8E00DC43232282
:10246000FE006384E71F83A2C700DC43AA96814E67
:102470002322FE00894F1303500A6306FF0683A838
:10248000C7009387480323A01601DCC283A78804F2
:1024900023A6F6019CC683A7C8029CCA83A7080589
:1024A00023AC0600DCCA03A8080383470800639630
:1024B0006710C287850703C70700B3850741E30B91
:1024C00067FE93D72500C207C183239EF600850EC1
:1024D00093860602638B120F83274E00DC43232270
:1024E000FE00E31EFFF88327CE002322FE0041BF3B
:1024F0008327CE1197EE0100938E8E32DC4317E7CF
:102500000100232DF7306384D71383AFC700DC436A
:102510003307D500014397E6010023A1F6300D4FA4
:1025200089429308500A6387D707C8479307450332
:1025300008C35CC33C452326E7011CC75C551CCB84
:102540001C5599C3232657003C49232C07005CCB1C
:10255000032805038347080063951705C28785078D
:1025600083C60700B3850741E38B16FF93D7250089
:10257000C207C183231EF700050313070702638AFE
:10258000AF028327CE11DC4397E6010023A8F6288B
:10259000E39DD7F983274E1297E6010023A0F62882
:1025A00069B78147231EF700050313070702E39A63
:1025B000AFFC1A94E31C06D225BB8147239EF6008C
:1025C000850E93860602E39912F117EE0100130EB1
:1025D0002E1383274E10769493165400E38307D06E
:1025E0001DB30147239EE700850E93870702E397FB
:1025F00012E597E701009387670003AE0700769422
:102600009316540083270E00E38607CCA1B58147BB
:10261000239EF600850E93860602E39E12D783273B
:102620008E11769493165400E38107CCD1B583279D
:102630004E1217E701002323F71EC1BD83270E1199
:1026400017E701002322F71CE1B98327CE002322DC
:10265000FE0011BD8326CE002322DE00B5B37971C2
:1026600026D24AD04ECE52CC56CA5AC85EC606D6DC
:1026700022D497E901009389A9F517E9010013090C
:10268000290817EA0100130A2AF697EA0100938A3B
:102690006AF797EB0100938BEBF597E401009384C5
:1026A000A4F5054B21A883A7090003244910850739
:1026B00017E70100232EF7F05D3011E89C40E5F7A5
:1026C00083270900E37CFBFEEFD05FD4C5BF7370A6
:1026D000043083270A00B9E383270911C047130593
:1026E0004400EFD0FFE883A70B00FD1717E70100B8
:1026F0002322F7F09C40FD1717E70100232EF7EE89
:1027000083270A0089C783A70A00FC4385E308588A
:10271000EF1050042285EF10F0034DB703A70A0015
:1027200083A70A007C4385077CC37DB703A70A0003
:1027300083A60A007C43FD177CC3FC42E9FB73605F
:102740000430F1B797E70100938787E89C43DDE702
:10275000411106C622C426C297E7010023A207E85A
:1027600017E70100130707EA1C43B7A6A5A5938640
:10277000565A9C5B8C43639BD500D0436318B600CC
:1027800094476395C600DC476388D70008430C4331
:1027900093854503EF20007417E70100130707E551
:1027A000144317E401001304A4F511A81C43A9CF96
:1027B0001C43FD1797E6010023AAF6E21443939702
:1027C0002600B6978A07A2979C43EDD30843931738
:1027D0002500AA978A073307F4005443A107A2975C
:1027E000C44244C36385F402DC44B240224417E788
:1027F00001002329F7E0924441018280854717E7D1
:102800000100232FF7DC82807370043001A0C440E4
:10281000D145EF50201E229544C1F9B701114AC895
:1028200006CE22CC26CA4EC62A897370043097E49D
:102830000100938464DB9C4017E40100130484DCF2
:10284000D9E76314090003290400930949004E8560
:10285000EFD01FD28327890289C713058901EFD0E2
:102860003FD1CE8517E50100130505FBEFD0DFCB87
:102870009C4081C71C40FC43ADE31C40638B270791
:102880009C409DCF737004309C40C1EB97E70100E2
:10289000938707D79843184325EBFD5717E70100A7
:1028A000232AF7D29C4089CF1C40FC4391CB18408F
:1028B00014407C43FD177CC3FC4299E373600430F1
:1028C000F2406244D2444249B249056182801840D4
:1028D0001C407C4385077CC3ADB7184014407C4343
:1028E000FD177CC3FC42D1FB736004301C40E399AC
:1028F00027F99C40A1C397E70100938767CD9C43CC
:10290000ADCB7370043001A09C43DC47DC47DC4353
:1029100017E701002320F7CC71B718401C407C4317
:1029200085077CC397E70100938787CD98431843B9
:102930002DD7D9BF97E701009387C7CB17E70100D1
:10294000130707DC9C4303278711631DF700F24040
:10295000624497E7010023A707CAD2444249B2491B
:10296000056182806244F240D2444249B249056125
:10297000D1BB6244F240D2444249B24905616FD0B2
:10298000FFA83DC9411126C297E40100938484C782
:102990004AC02E898C4006C622C4E105EFD05FBA3A
:1029A00088401105EFD0DFBCFD57630AF90497E7B3
:1029B00001009387E7C3804398409C434A9440C3F7
:1029C000636CF40497E70100938787C388438C40C6
:1029D0009105EFD0FFB697E701009387A7BF9C430F
:1029E0006376F40097E7010023A687BEB240224435
:1029F00092440249410182807370043001A08C40EE
:102A00002244B2409244024917E501001305C5E093
:102A1000910541016FD05FB197E70100938707BE31
:102A2000884322448C40B2409244024991054101BE
:102A30006FD01FB111C997E70100938767B99C4315
:102A400099E77370043001A07370043001A0411144
:102A500026C297E401009384E4BA9840AE878C4084
:102A6000B7060080D58F06C622C41CCFE10532848C
:102A7000EFD09FAB88401105EFD09FAFFD57630E9D
:102A8000F40097E701009387A7B68843B2409244C9
:102A90002295224441016F5020088C402244B240CC
:102AA000924417E50100130525D7910541016FD028
:102AB000BFA725CD411126C297E40100938484B4B9
:102AC0004AC02E898C4006C622C4E1053284EFD06C
:102AD000BFA588401105EFD0BFA98547630AF4045C
:102AE00097E701009387C7B0804398409C434A947E
:102AF00040C3636CF40497E70100938767B0884391
:102B00008C409105EFD0DFA397E70100938787AC56
:102B10009C436376F40097E7010023AD87AAB24097
:102B2000224492440249410182807370043001A022
:102B30008C402244B2409244024917E5010013053B
:102B4000A5CD910541016FD03F9E97E70100938786
:102B5000E7AA884322448C40B2409244024991053E
:102B600041016FD0FF9D411106C622C426C25C45BB
:102B7000C04735CC930484012685EFD07F9F97E72B
:102B800001009387E7A49C43B5E79304440026859E
:102B9000EFD01F9E97E70100938747A558549C43A9
:102BA00063F6E70097E7010023A2E7A49317270045
:102BB000BA978A0717E50100130585B4A6853E95E7
:102BC000EFD09F9697E701009387C7A39C43585483
:102BD0000145DC5763F8E700854717E7010023212B
:102BE000F7A00545B24022449244410182807370AF
:102BF000043001A0A68517E50100130565BFEFD0DD
:102C0000BF92C9B797E701009387879C9C4381E7F0
:102C10007370043001A0411106C622C426C2B70752
:102C200000804045CD8F1CC12DC4EFD07F9493040C
:102C300044002685EFD0DF9397E701009387079B39
:102C400058549C4363F6E70097E7010023A0E79AF6
:102C500093172700BA978A0717E50100130545AABD
:102C60003E95A685EFD05F8C97E701009387879903
:102C70009C4358540145DC5763F8E700854717E744
:102C80000100232FF7940545B240224492444101AC
:102C900082807370043001A011CD97E70100938703
:102CA000E793984397E70100938787949C4318C163
:102CB0005CC182807370043001A055C1D1CD411137
:102CC00006C622C42A877370043097E801009388EF
:102CD000A89183A7080091CB97E70100938787927B
:102CE00094439C43FC428507FCC217E30100130395
:102CF00023909C4103260300FD560144638FD702B5
:102D000017EE0100130E8E8D03250E000328070019
:102D100054436305A80005446371D6023308D640C6
:102D20000544637CF80003250E00918F0326030001
:102D3000B6979CC108C350C3014483A7080081CB48
:102D400097E701009387078C9C43FC4381EF228522
:102D5000B2402244410182807370043001A073703C
:102D6000043001A0EF409061DDB7854717E701000F
:102D70002328F786828019C16845828001458280B8
:102D800011C16CC5828097E701009387A7878843AC
:102D9000828097E70100938727859C43054589CB6F
:102DA00097E701009387C78288431335150006050E
:102DB000828031CD011126CA97E401009384848476
:102DC0009C4006CE22CC4AC84EC65855DC57637983
:102DD000F7021C4D63C707009C40D457A947958F45
:102DE0001CCD93172700BA97584917E9010013091A
:102DF00029918A07CA97630DF7009C40DC575CD580
:102E0000F2406244D2444249B249056182808280E4
:102E1000930945002A844E85EFD08FF59C4017D743
:102E200001001307A77C1843DC575CD46376F700D6
:102E300017D70100232CF77A139527003E9562449B
:102E40000A05F240D244CE854A95B249424905610D
:102E50006FD08FED19CD411106C622C426C297D777
:102E600001009387277A80436307A40073700430BE
:102E700001A0014582807C4881E77370043001A085
:102E800054543848FD177CC86383E60099C7014550
:102E9000B24022449244410182809304440026853A
:102EA000EFD00FED284897D70100938727749843F8
:102EB000A947898F48D41CCC6376A70097D7010017
:102EC00023A6A772D145EF40F03297E70100938720
:102ED00027833E95A685EFD02FE5054555BF737036
:102EE000043097D70100938727709C4391CB97D7E5
:102EF00001009387277198439C437C4385077CC3DB
:102F0000828097D701009387276E9C438DC397D704
:102F100001009387276F9843784311CB98439443DC
:102F20007C43FD177CC3FC4299E3736004308280CC
:102F300097D701009387076D904394439843A9471F
:102F4000D456084E958F1CCF828097D70100938767
:102F5000676B984309C79443F84A0507F8CA884342
:102F6000828079714AD006D622D426D24ECE2A89C2
:102F70007370043097D40100938404679C4017D485
:102F8000010013042468BDE31C40BC4F89E71C40CA
:102F90000547F8CFD1E19C4081C71C40FC43F1EBD1
:102FA000737004309C408DEF1C40A84F11C5630422
:102FB00009021C4023AC07041C4023AE07049C40BC
:102FC00081C71C40FC438DEBB250225492540259ED
:102FD000F2494561828018403C4FFD173CCFE9BF64
:102FE00018401C407C4385077CC37DBF18401C40B3
:102FF0007C4385077CC349BF184014407C43FD17C0
:103000007CC3FC42F1F373600430B25022549254FA
:103010000259F2494561828008402EC61105EFD061
:103020002FD5B245FD576380F50697D701009387EA
:10303000275C83A9070018409C43AE9923223701DF
:1030400063ECF90497D701009387875B88430C40B2
:103050009105EFD0EFCE97D701009387A7579C43F8
:1030600063F6F90097D7010023A63757EFD00FBAC0
:103070001DB7184014407C43FD177CC3FC428DF300
:103080007360043031BF0C4017D501001305C578BB
:103090009105EFD06FC9D9BF97D701009387075625
:1030A00088430C409105EFD0AFC9C9B779714AD0B8
:1030B0004ECE06D622D426D252CC2E89B289737037
:1030C000043097D40100938424529C4017D401000B
:1030D00013044453F9EF18408947784F630CF70005
:1030E0001C401345F5FFB84F798DA8CF1C4005470C
:1030F000F8CFADE69C4081C71C40FC43F5E37370FC
:1031000004309C40B1E7638609001C40BC4F23A0FB
:10311000F900184085470145784F630BF7001C40C4
:103120001349F9FF0545B84F3379E90023AC27056A
:103130001C4023AE07049C4081C71C40FC43C1E3F4
:10314000B250225492540259F249624A4561828037
:1031500018401C407C4385077CC375B7084036C6C1
:103160001105EFD0EFC0B246FD576385F60897D73B
:1031700001009387E74703AA070018409C43369A4B
:10318000232247016363FA0897D7010093874747D3
:1031900088430C409105EFD0AFBA97D701009387D1
:1031A00067439C436370FA0697D7010023A4474303
:1031B00091A818401C407C4385077CC329BF184058
:1031C00014407C43FD177CC3FC42BDFB736004309C
:1031D000B250225492540259F249624A45618280A7
:1031E000184014407C43FD177CC3FC4289FB73608C
:1031F000043031B70C4017D501001305E561910586
:10320000EFD08FB2EFD08FA0F5B597D7010093879D
:10321000E73E88430C409105EFD08FB2E5B751C12E
:10322000411106C622C426C24AC07370043097D426
:1032300001009384643B9C40B9EB99C23C4D9CC215
:10324000B2878946704D74CD2E872A846386D7064F
:1032500063FCF6048D456387B70091456395B7001D
:103260006300D60C38CC8547630FF60405449C40B8
:1032700081CB97D701009387E7389C43FC43A9E3B0
:103280002285B2402244924402494101828097D76C
:1032900001009387273798439C437C4385077CC371
:1032A00069BF7370043001A08546E39ED7FA3C4D98
:1032B00033E7B70038CD45BF3C4D85073CCD65B7FA
:1032C000EF40D00B75BF130944004A85EFD04FAAD9
:1032D00097D701009387873148549C4363F6A70032
:1032E00097D7010023A4A730D145EF40A07097D70E
:1032F00001009387E7403E95CA85EFD0EFA21C54AA
:1033000081C77370043001A097D701009387872F7E
:103310009C435854DC57E3FBE7F4EFD02F8FB9B749
:103320000144B1B739CD011122CC26CA4AC84EC6D4
:1033300052C456C206CEBA89368AB2842E892A84ED
:10334000EFD0AF98AA8A63050A003C4C2320FA000C
:10335000784C89477CCC6389F40263F4970C8D46E2
:103360006387D40091466396D400630AF70A232C3E
:1033700024058547631EF7061C5499CB73700430EF
:1033800001A07370043001A03C4C85073CCCD5B73C
:1033900097D701009387C7239C43ADEB9304440068
:1033A0002685EFD0EF9C97D70100938727244854B8
:1033B0009C4363F6A70097D7010023A9A722D14514
:1033C000EF40406397D7010093878733A6853E95EA
:1033D000EFD08F9597D701009387C7229C4358540D
:1033E000DC5763F7E70063850900854723A0F900F0
:1033F00005445685EFD00F8D2285F2406244D244B9
:103400004249B249224A924A056182809305840169
:1034100017D501001305C53DEFD00F9165BF0144DD
:10342000C9BF8547E397F4F43C4C33E92701232CCB
:10343000240581B74DC1011122CC26CA2A844EC66B
:1034400006CE4AC8AE84EFD04F888947744C7CCCF6
:103450003C4C0547AA8985073CCC6395E6061C547D
:1034600081C77370043001A097D701009387471676
:103470009C43ADE7130944004A85EFD06F8F97D77F
:1034800001009387A71648549C4363F6A70097D77B
:10349000010023ADA714D145EF40C05597D70100D7
:1034A00093870726CA853E95EFD00F8897D70100EE
:1034B000938747159C435854DC5763F5E70099C040
:1034C00085479CC06244F240D24442494E85B2498D
:1034D00005616FC03FFF7370043001A09305840144
:1034E00017D501001305C530EFD00F84C1B7AA87E7
:1034F00029C57370043017D701001307E70E144372
:103500009DE2F04F894601456315D60023AE0704BE
:1035100005451C4381CB97D701009387A70E98439D
:10352000784315E3828097D601009386A60D9042DA
:1035300094427442850674C2E9B797D70100938715
:10354000670C9C437DB7984394437C43FD177CC331
:10355000FC42E9FB7360043082805D71A6C2CAC080
:1035600052DC56DA5AD85ED686C6A2C44EDE62D483
:1035700066D26AD017D901001309C90917DB010007
:10358000130B8B0897D401009384440897DA010049
:10359000938A0A08054AA54B8327090098436301CB
:1035A0000712DC4783A90700EFE06FF6EFE02FF783
:1035B00083270B002A8C6362F50A97D7010023A5A5
:1035C000A70401466370351B8840B3858941EFD05D
:1035D000DFBDEFE0DF9863010512884081460146B8
:1035E0002C00EFD0EFEB4DD9A247E3C807FEC2494C
:1035F00083A7490189C713854900EFC07FF7EFE032
:103600000FF283270B002A8C636DF508A24717D7AA
:103610000100232B87FFE3E2FBFCB317FA0013F74B
:103620000721631A071613F7770C6318071E93F721
:103630000702C5D74E85EF00F01145B7DC47C047FC
:1036400083AC0700930944004E85EFC07FF25C50C5
:10365000228582975C4C6384470B8327090098433B
:1036600071FF03A70A0097D6010023AF86F997D60A
:10367000010023AFF6F897D7010023ADE7F8EFE09C
:103680001F8EA1BFDC47C04703AD0700930C440069
:103690006685EFC0FFED5C50228582975C4C6386A7
:1036A000470983270900984371FF03A70A0097D6AB
:1036B000010023AFF6F497D7010023ADE7F4B9B7C3
:1036C000EFE0EFE4EFE0AFE583270B002A8CE36641
:1036D000F5F883A70A00884081499043B385894162
:1036E00017D70100232287F313361600EFD0FFAB64
:1036F000EFE0FF86E31305EEEFC05FD1F9BD1C4C90
:10370000CE85E69763E9FC049C4089CF02CA66CC6B
:1037100022CEEFF00FE88840814601464C08EFD0FA
:103720000F8805FD7370043001A01C4CE685EA97F4
:10373000636CFD049C4089CF02CA6ACC22CEEFF0B4
:103740004FE58840814601464C08EFD04F8531F95E
:103750007370043001A0032509005CC000C8EFC0ED
:103760003FDEE5BDEFE0AFFF83270900DC47C04740
:10377000930C44006685EFC0BFDF5C4C638F47034A
:103780005C502285829791BD032509005CC000C86A
:10379000EFC01FDB39B7B24723ACF900A5CFE297E2
:1037A00023A2F90023A8390193854900636FFC0423
:1037B00003A50A00EFC0DFD80DB51C4C00C8338745
:1037C000F90058C0636DEC02330C3C416363FC02AA
:1037D0009C4089CF02CA4ECC22CEEFF08FDB8840CE
:1037E000814601464C08EFC09FFB59F973700430C5
:1037F00001A003A50A00E685EFC09FD451B70325B9
:103800000900E685EFC0DFD3A5BF03250900EFC09F
:103810003FD3E1B37370043001A0B24783A689019E
:1038200023A839013387D70023A2E9006364EC049D
:10383000B307FC4063EBD70483A749024E85829708
:1038400083A7C901E39B47D983A68901B247984062
:10385000B69711CF02CA3ECC4ECEEFF08FD3884040
:10386000814601464C08EFC09FF3E31805D67370FC
:10387000043001A06374FC00E370F7FC0325090029
:1038800093854900EFC0DFCB89BB03A50A00938570
:103890004900EFC0FFCA91B3411122C406C626C237
:1038A0004AC017D40100130464D6EFF04FE31C4064
:1038B00095CBEFF00FE51C409DC38148014881473F
:1038C000094781461306004097D50100938585B6C8
:1038D000170500001305A5C8EFD05F9A39E973708A
:1038E000043001A017D90100130949F44A85EFC03B
:1038F0001FC297D401009384A4F42685EFC03FC172
:103900000146B145114597D7010023A527D197D787
:10391000010023AF97CEEFC07FDB17D7010023272D
:10392000A7CE11CD97D50100938545B0EFD0AFFC60
:1039300049B7B240224492440249410182807370E7
:10394000043001A0A5C9797156CAAA8A1305C0021C
:1039500022D426D24AD04ECE52CC06D65AC85EC603
:103960003A89B689328AAE84E9212A8405C9EFF002
:103970000FD797D70100938767C99C439DCFEFF07E
:103980004FD8130544002320540104CC232E4401B6
:103990002320340323222403EFC0BFB82285B25072
:1039A000225492540259F249624AD24A424BB24BD3
:1039B000456182807370043001A097DB0100938B16
:1039C000EBE65E85EFC0BFB417DB0100130B4BE7DE
:1039D0005A85EFC0DFB30146B145114597D70100C5
:1039E00023AA77C397D7010023A467C3EFC01FCED4
:1039F00017D70100232CA7C001C997D501009385D3
:103A0000E5A2EFD04FEFA5BF7370043001A039C518
:103A1000011122CC06CE26CA17D40100130404BF1C
:103A2000832804002A88014563850802BA842EC2CF
:103A3000368732C442C6954663C5B602EFF06FB50D
:103A40008947630BF5020840814601464C00EFC0F0
:103A50001FD5F2406244D244056182807370043005
:103A600001A04C0081463A864685EFD08F88F2400F
:103A70006244D244056182800840814626864C001B
:103A8000EFC0FFD1F9B719C10841828073700430CB
:103A900001A001E57370043001A0411106C622C4E3
:103AA0002A84EFF0CFC348483334A000EFF06FC54D
:103AB0002285B24022444101828001E573700430C6
:103AC00001A0411122C42A8406C6EFF04FC1005064
:103AD000EFF02FC3B240228522444101828001E5EC
:103AE0007370043001A0411122C426C22E84AA841E
:103AF00006C6EFF0CFBE80D02244B24092444101CE
:103B00006FF02FC04111714522C406C61D262A84BC
:103B100011C5232005001105EFC07F9F2285B2400B
:103B200022444101828001CDB70700FFED8F81C79C
:103B30007370043001A099E57370043001A07370B4
:103B4000043001A0011122CC4AC84EC652C456C24C
:103B500006CE26CABA893689B28A2E842A8AEFF01E
:103B60004FA311E5638509007370043001A0EFE0F5
:103B70000F9A83240A00B37794006316090295C74D
:103B800063870A009347F4FFE58F2320FA00EFE0F4
:103B90000FBDF240624426854249D244B249224ACE
:103BA000924A05618280E30DF4FCE38209FEB3359D
:103BB0005001E20563050900B7070004DD8D4E865C
:103BC000C18D13054A00EFE0FFE6EFE04FB919E1C0
:103BD000EFC0DF83EFF0CFB593176500AA8963D8F4
:103BE0000700B7040001FD14B3F499005DB7EFF0CE
:103BF0000FAF83290A00B3773401631E090089CB14
:103C000063880A009347F4FFB3F737012320FA00D3
:103C1000EFF02FAFF9B7E31DF4FEDDB701C9B70729
:103C200000FFED8F99C77370043001A073700430EA
:103C300001A0411122C42A8406C626C24AC02E8988
:103C4000EFF0EFA904409345F9FFB3F795001CC0CE
:103C5000EFF02FABB2402244268502499244410145
:103C60008280411122C42A8406C6EFC01F8600400C
:103C7000EFC05F85B240228522444101828009C99C
:103C8000370700FFB3F7E50099C77370043001A050
:103C90007370043001A06F303070B70700FFF18FF0
:103CA00081C77370043001A001E67370043001A075
:103CB000011122CC4AC84EC652C406CE26CA368945
:103CC000AE892A8A3284EFF0CF8C21E163050900A6
:103CD0007370043001A0EFE08F8383240A00CE8547
:103CE0005285B3E49900613FB37794006307F4060B
:103CF00083240A00EFE0AFA6F240624426854249E1
:103D0000D244B249224A05618280EFE04F80832489
:103D10000A00CE855285B3E434019537B3F78400A9
:103D2000638D8702E30609FCB70500054A86C18D4D
:103D300013054A00EFE01FD0EFE06FA219E1EFC0DA
:103D4000EFECEFF0EF9E93176500AA8463DF0700A6
:103D5000B7070001FD17FD8C45B783270A00134400
:103D6000F4FFE18F2320FA0071B7EFF04F9783241F
:103D70000A00B3779400639787009347F4FFE58FB9
:103D80002320FA00EFF0EF97E1B7411122C406C6F5
:103D90002A8426C2EFD0BFF75C4085C3084893044D
:103DA000C4006316950015A0084863009502B70586
:103DB0000002EFE03FE55C40E5FB2285612A2244FA
:103DC000B240924441016FE08F997370043001A0BA
:103DD00009C9370700FFB3F7E50099C773700430CE
:103DE00001A07370043001A06F30105B01C9B707E8
:103DF00000FFED8F99C77370043001A07370043019
:103E000001A0411122C426C206C62A84AE84EFF066
:103E10000F8D184093C7F4FFF98F1CC02244B240A5
:103E2000924441016FF0EF8D19C1084D8280014528
:103E30008280411122C406C62A84EFD05FED97C765
:103E400001009387677D9C43A1EBE56717D70100CD
:103E5000130787A0F11797C6010023A5E67C17C7B3
:103E60000100232FF77A17D701002329F79E97C760
:103E700001009387A77A17D70100232FF79C854766
:103E800017C701002322077A17C7010023280778E4
:103E900017C701002322F77819E8EFE04F8CEF10E5
:103EA000E00201442285B240224441018280130590
:103EB000840093773500C1EFE5671307F5FFE91735
:103EC000E3EDE7FC97C601009386C6759C4229A0E6
:103ED000984311C7BE86BA87D843E36BA7FE17C7BE
:103EE00001001307A773E38AE7FA98434146138456
:103EF000870098C2D843B306A7406378D6023388B8
:103F0000A7002322D800C8C38325480097C6010014
:103F10009386467111A0BA8698425043E36DB6FE6F
:103F20002320E80023A00601D84397C70100938708
:103F300027739C43998F17C701002323F772EFE083
:103F40000F8231DC2285B240224441018280719986
:103F500011059DB729C9411122C406C62A84EFD094
:103F60001FDB930584FF0326C4FF17C70100130757
:103F7000676B11A03E871C43D443E3EDC6FE232CA0
:103F8000F4FE0CC397C701009387876D984383277E
:103F9000C4FF2244B240BA9717C701002322F76C2E
:103FA00041016FD0DFFB828097C701009387476B89
:103FB0008843828082803367B5000D8BAA871DE716
:103FC0009308D6FFAA982A87AE866371150303A8C3
:103FD000060011079106232E07FFE36A17FF934798
:103FE000F5FFC697F19B9107BE95AA972A9663F3B2
:103FF000C70A9386450013884700B3B6D70033B885
:10400000050133E7F50093C61600134818000D8B21
:10401000B3E6060113371700758F330EF64093860B
:10402000170029CF1337AE0031EB13532E002E8823
:10403000BE860147832808000507110823A0160142
:104040009106E36967FE1377CEFFBA95BA976302CC
:10405000EE0483C60500138717002380D700637A18
:10406000C70283C6150013872700A380D700637299
:10407000C70203C725002381E7008280B307F6400B
:10408000AE97850503C7F5FF8506238FE6FEE39A05
:10409000F5FE82808280B367C5008D8BB308C500B2
:1040A000E9C36371150FB307A0408D8B13873700E9
:1040B000954693F5F50F130815003383A8407D1638
:1040C0006373D70015476363E60CD5CF2300B500B3
:1040D0000547638DE700A300B5000D4713082500D1
:1040E0006396E700130835002301B5001396850099
:1040F0004D8E13970501518F3303F340939685013D
:10410000D98E13562300AA97014794C30507910738
:10411000E36DC7FE1377C3FFB307E8006307E30649
:104120002380B70013871700637C1703A380B700B1
:1041300013872700637617032381B700138737009F
:1041400063701703A381B70013874700637A1701D1
:104150002382B7001387570063741701A382B70047
:10416000828093F5F50F13978500D98D139705017C
:104170004D8FE37715FFAA87910723AEE7FEE3EDA6
:1041800017FF828082802A8895B78280AA8749BFDC
:10419000834705002A8799C7050583470500EDFF7A
:1041A000198D82800145828005058347F5FF8505CD
:1041B00003C7F5FF91C7E389E7FE3385E7408280B7
:1041C0008147E5BFAA87850503C7F5FF8507A38F4C
:1041D000E7FE75FB82808346050093070002639724
:1041E000F600050583460500E38DF6FE938756FD30
:1041F00093F7D70F85C7AA87814585CE01458507E7
:10420000138606FD1317250083C607003A95060599
:104210003295F5F699C13305A0408280938536FD2D
:104220008346150093B5150093071500E1FA014583
:10423000D5B7014582809C412380A7009C4185071A
:104240009CC1828097C601009386463E9C421757C8
:1042500003001307276313861700BA972380A7006C
:1042600097C5010023A4C53CA9476308F50093073F
:1042700000046305F6000145828075DE370610F004
:1042800005078347F7FF2320F6F09C42FD1797C5EB
:10429000010023ADF538EDF7014582804D712322F1
:1042A000911423202115232A51132324811323261B
:1042B000111423248114232E3113232C411323287A
:1042C000611323267113232291132320A113232E7C
:1042D000B111AA842E8932C6130C5002A54A834715
:1042E000090063808703B9CB804011A0A1CB2300D4
:1042F000F40080400509050480C083470900E39766
:1043000087FF0346190093081900C686130D0002A3
:10431000FD597D5A0148130550059307D6FD93F7C3
:10432000F70F138916006363F52A17C701001307F7
:1043300067CD8A07BA979C43BA9782878320C114B6
:104340000324811483244114032901148329C113F4
:10435000032A8113832A4113032B0113832BC112D8
:10436000032C8112832C4112032D0112832DC111C4
:1043700071618280A14C02C4854763D50715B2479D
:104380008040938B770093F68BFF03AB060083A9E5
:104390004600938786003EC6668681465A85CE854E
:1043A000EF10907E2AC8814763853723930D410122
:1043B000854B668681465A85CE85EF10301F814633
:1043C00066862A8BAE89EF10307CA24723A0AD0011
:1043D00093861B00910D63843701B68BD9BFE37EB2
:1043E0009BFF63DD4601A2872380A70180407D1AE1
:1043F000930714009CC03E84E3C846FF93962B00AD
:104400001C08BE9631A8938777052300F4008040EE
:10441000FD1B93871B00050480C0F116E351F0ECEF
:104420009C42E3E2FAFE93870703C5B79C409306DC
:10443000000332472380D7009C4093064700C14CBD
:104440001386170090C013068007A380C700804022
:1044500002C4BA87050480C003AB0700814936C691
:1044600025BFB24783AC0700938B470063840C1CC5
:10447000635F40199307D0026319FD1683C70C00D0
:1044800085C363DC09189440850C7D1A2380F600EF
:104490008040050480C083C70C00E5F7635D4001E0
:1044A0008040930700022300F40080407D1A050439
:1044B00080C0E31A0AFE5EC61DB502C48547A94C3A
:1044C000E3CF07EBB24780409386470071B703C63E
:1044D0001600CA8699B59C40930650022380D700E7
:1044E0008040050480C0E5BBC14C02C471B5B24731
:1044F00003C61600CA8683A9070091073EC6E35E7D
:104500000AE04E8AFD5911BD03C61600130DD002F4
:10451000CA8621B59347FAFFFD8703C61600337A92
:10452000FA00CA86DDBB03C61600130D0003CA8657
:10453000EDB383C51600930906FDCA86938705FD72
:104540002E86E3EEFAFA93972900BE99850686092E
:10455000AE9983C50600938909FD938705FD2E86D4
:10456000E3F3FAFE69BF32479C40144311073AC691
:104570002380D7008040050480C095B3854763D36E
:10458000070BB24793867700E19A938786003EC671
:1045900083A946009C4263DC090A94401306D002BA
:1045A000B307F0402380C6008040B336F000B30963
:1045B0003041050480C03E8BB389D940A94C02C468
:1045C000E1BB03C616000508CA8681BB9C4046892C
:1045D00021B7E37D9BDD8547814B8546E3C547E1F8
:1045E00031BD97CC0100938C6CE5CE856685EF10CC
:1045F0002024330AAA40635C400180402300A401C8
:1046000080407D1A050480C0E31A0AFE014A83C770
:104610000C00E38207EAE3C809E6FD197D57E3943D
:10462000E9E6ADBDB247938647009C4336C693D9B1
:10463000F74195B7635640019307D002E313FDFAA3
:1046400097CC0100938C8CDF930780021DBD3E8BBD
:10465000A94C02C4804089B34D71232E3113B70990
:1046600000409387F9FF2324811423229114232CE3
:104670004113232A51132326111423202115232803
:1046800061132326711323248113232291132320E2
:10469000A113232EB1112A8A2EC417C401001304BA
:1046A000E4F8975A0300938AEA1D97C401009384A3
:1046B000E4AA3EC693055002294513080004B70634
:1046C00010F083470A006386B704C1C71840050A83
:1046D00013061700569797C8010023A9C8F42300B2
:1046E000F7006382A706E31E06FD175703001307B2
:1046F000671905078347F7FF23A0F6F01C40FD1755
:1047000017C601002324F6F2EDF783470A00E39E63
:10471000B7FA83461A0013051A002A87930B000282
:104720007D5B7D5C014893055005A5489387D6FDC8
:1047300093F7F70F130A170063E7F5348A07A69774
:104740009C43A6978287175703001307A71355F2B8
:104750008DBF8320C11403248114832441140329B1
:1047600001148329C113032A8113832A4113032BC4
:104770000113832BC112032C8112832C4112032DB0
:104780000112832DC11171618280A14C014D8547B9
:1047900063DB0719A2479D07E19B83AD070003ABCD
:1047A0004700138787003AC4668681466E85DA859E
:1047B000EF10903D2AC863066D3513094101854904
:1047C000668681466E85DA85EF10405E6686814694
:1047D000AA8D2E8BEF10503B2320A90085091109CB
:1047E000E3106DFFE3FE9DFD13060004B70610F015
:1047F00063D189031C4013871700D69797C5010022
:1048000023A6E5E223807701630CC7047D1CE3C384
:1048100089FFB2476800A548B386F9008A061C08DC
:10482000BE96294813030004370610F0E384A6E877
:104830009C429305000363F4F8009305700518404B
:10484000AE9793051700569717CE01002320BEDEC2
:104850002300F7006380072B638C6526F116F9B7F8
:10486000175703001307070205078347F7FF23A025
:10487000F6F01C40FD1797C5010023A9F5DAEDF706
:104880007D1C71B71C40130600041387170097C5E1
:10489000010023ADE5D8B386FA0093050003238019
:1048A000B6006300C73E890797C6010023A0F6D86B
:1048B0005697930680072300D70017570300130766
:1048C00067FCB70610F0639EC70005078347F7FF34
:1048D00023A0F6F01C40FD1717C601002328F6D4CC
:1048E000EDF7A247C14C014D91072247014B832DA3
:1048F00007003EC455BDA24783AC0700138947009B
:10490000638F0C3A635480219307D002639EFB2E81
:1049100003C70C00BA856310072025AC8547A94C56
:10492000014DE3C907E7A2479107C1B7A2478346F4
:104930001700528703AB070091073EC4E3580CDE13
:104940005A8C7D5BE5B383461700930BD0025287E8
:10495000F1BB9347FCFFFD8783461700337CFC00C7
:104960005287E9B383461700930B000352877DBB40
:1049700003461700138B06FD5287930706FDB28688
:10498000E3EEF8FA93172B00DA9705078607B2973C
:1049900003460700138B07FD930706FDB286E3F37A
:1049A000F8FE69BFA2451C4029469841938617002E
:1049B000D69717C50100232BD5C62380E70013899E
:1049C00045006301C72A930700046387F6204AC4A1
:1049D000D5B1854763DF0729A24713877700619B1D
:1049E000930787003EC4032B47001C43635B0B30D7
:1049F0001840130600049306170097C5010023A76B
:104A0000D5C256979305D0022300B7006388C62C01
:104A1000B307F0403337F000330B6041BE8D330BEA
:104A2000EB40A94C014D49B3834617000508528756
:104A3000F5B9834617005287D5B91C409306000488
:104A40001387170017C601002322E6BED697130668
:104A500050022380C700E31FD7C417570300130772
:104A600067E2B70610F005078347F7FF23A0F6F0CB
:104A70001C40FD1717C60100232AF6BAEDF71DB931
:104A8000C14C014D29B31C40930600042A8A1387A8
:104A9000170017C60100232BE6B8D697130650025D
:104AA0002380C700E318D7C017570300130787DD1B
:104AB000B70610F005078347F7FF23A0F6F01C4068
:104AC000FD1717C601002323F6B6EDF72A8ADDB6D7
:104AD00017570300130707DB05078347F7FF23205A
:104AE000F6F01C40FD1797C5010023A1F5B4EDF7C2
:104AF000F1162DBB175703001307C7D8F1FDF116A8
:104B000035B3E3FC9DCB8549C5B1014C03C70C000F
:104B1000BA85E30E07EAFD58294513080004B706D5
:104B200010F063570B0A1C4013861700D69717C363
:104B30000100232DC3AE2380E7006384A506630430
:104B40000609850C03C70C007D1CBA8579FBE35070
:104B500080E91C409305000213060004B70610F01C
:104B600021A07D1CE3050CE613871700D697238050
:104B7000B70017C50100232BE5AABA87E313C7FEC8
:104B800017570300130707D005078347F7FF23A034
:104B9000F6F01C40FD1717C501002329F5A8EDF715
:104BA000C9B7175703001307E7CD41DE0507834751
:104BB000F7FF23A0F6F01C40FD1717C601002327BE
:104BC000F6A6EDF7BDBF175703001307A7CBF9BF34
:104BD0007D1BE31A1BF5A5BF17570300130787CAF0
:104BE000B70610F005078347F7FF23A0F6F01C4037
:104BF000FD1717C60100232BF6A2EDF74AC45DBCD2
:104C000097CC0100938C8C83DA856685EF00504247
:104C1000330CAC40E35C80EF1C4013060004B70685
:104C200010F021A07D1CE3020CEE13871700D6972D
:104C30002380770197C5010023AAE59EBA87E31375
:104C4000C7FE175703001307E7C305078347F7FF9E
:104C500023A0F6F01C40FD1797C5010023A8F59C82
:104C6000EDF7C9B7175703001307C7C1B5FA4AC410
:104C700091B4A247138747009C433AC413DBF74122
:104C8000B5B3175703001307E7BFB70610F00507C2
:104C90008347F7FF23A0F6F01C40FD1717C601005D
:104CA0002326F698EDF7854717C701002320F798CC
:104CB00093078007175703002306F7BC1DB16356FF
:104CC00080019307D002E39DFBF297BC0100938C17
:104CD000EC76130780029305800235BD97560300DA
:104CE000938646BA370610F0850603C7F6FF2320E1
:104CF000E6F018407D1797C5010023A9E5926DF7EE
:104D000001BBBE8DA94C014D45B4B70710F023A0DF
:104D1000A7F201A03971130341022ED29A8506CE63
:104D200032D436D63AD83EDA42DC46DE1AC62D32C6
:104D3000F2400145216182805D711303810322D419
:104D40002AC632DC2A841A86680006D6BEC236DE3F
:104D5000BAC0C2C4C6C61ACEEFF04FD4B247238041
:104D600007003245B250018D225461618280B7073D
:104D700010F083A647F403A607F403A747F4E31A49
:104D8000D7FE8566938606FAB29633B6C600B3059B
:104D9000E60023A4D7F423A6B7F48280B70710F067
:104DA00003A747F403A607F483A647F4E31AD7FE44
:104DB0008566938606FAB29633B6C60023A4D7F466
:104DC000B305E60023A6B7F49307000873A04730A5
:104DD0008280411122C406C697C701009387878548
:104DE00017C401001304C48498431C401306F07CCC
:104DF000930647069387470697C5010023ACD582E3
:104E000097C5010023A6F5826346D600B24022442E
:104E1000410182801307478997C7010023ACE780CF
:104E2000EF00900A8547631FF50018408567938758
:104E3000F7760145E3DCE7FCC93D2244B24041017D
:104E40006FC0FFEB17B501001305C55FE1350945DC
:104E50006D3D2244B24041016FC07FEA17B50100A9
:104E6000130505606FF01FEB17B501001305C55F53
:104E70006FF05FEA411122C426C206C6856417B4EA
:104E800001001304E45E938784380100FD17F5FFE9
:104E90002285EFF03FE8C5BF01456F00006E41116C
:104EA00006C6EF007002054781476316E500B24071
:104EB0003E854101828017B501001305A558EFF02A
:104EC0007FE5B24089473E8541018280737004309E
:104ED00001A082807370043001A05D7197B701005A
:104EE000938787754EDE83A9070097B701009387E4
:104EF000E774CAC003A9070097B7010093874774F6
:104F0000A6C284434EC64AC826CAB247C245A2C4F6
:104F100052445AD82A8B3E8586C652DC56DA5ED673
:104F2000EF109016A285EF20602E2ACE814A17BA84
:104F30000100130A2A71B70B00804EC64AC826CA60
:104F40003245C2455244EF103014A285EF20002CA8
:104F50002ACC6245F245EF20606293050000EF2005
:104F6000201E634905026245F245EF20206183253A
:104F70000A00EF2020103325A00019E9E39F0AFA68
:104F800083570B008507C207C1832310FB0075B749
:104F9000854A65B76245F24533C5AB00EF20005E38
:104FA00083250A00EF20000D3325A000F9B75D71BD
:104FB00097B70100938747694EDE83A9070097B72B
:104FC00001009387A768CAC003A9070097B701002B
:104FD00093870768A6C284434EC64AC826CAB2470A
:104FE000C245A2C452445AD82A8B3E8586C652DC9A
:104FF00056DA5ED6EF10904EA285EF2020212ACE01
:10500000814A17BA0100130AEA63B70B00804EC643
:105010004AC826CA3245C2455244EF10304CA285D8
:10502000EF20C01E2ACC6245F245EF2020559305A3
:105030000000EF20E010634905026245F245EF20D1
:10504000E05383250A00EF20E0023325A00019E990
:10505000E39F0AFA83570B008507C207C183231019
:10506000FB0075B7854A65B76245F24533C5AB00AD
:10507000EF20C05083250A00EF10D07F3325A00019
:10508000F9B71D712AC613058002A2CCA6CACEC6E6
:10509000D2C4D6C2DAC05EDE62DC66DA6AD86ED608
:1050A00086CECAC8EFE0FFD897B701009387875A2A
:1050B00084432A8402C4A68D268DA68C268CA68BBA
:1050C000268BA68A268AA689930700003EC83ECA78
:1050D0003ECE7245A685EF20601308C07245424956
:1050E000EE85EF20A012CA85EF10007A2AC872451B
:1050F000EA85EF20A01148C072454249E685EF20BD
:10510000E010CA85EF1040782AC87245E285EF208A
:10511000E00F08C472454249DE85EF20200FCA85A2
:10512000EF1080762AC87245DA85EF20200E48C439
:1051300072454249D685EF20600DCA85EF10C074D4
:105140002AC87245D285EF20600C08C872454249D2
:10515000CE85EF20A00BCA85EF10007397B7010032
:105160009387474F2AC872458C43EF20200A97B790
:1051700001009387274E48C872458C434249EF206F
:10518000E008CA85EF10407097B701009387874CFD
:105190002AC872458C43EF20600797B701009387B8
:1051A000674B08CC72458C434249EF202006CA85E4
:1051B000EF10806D97B701009387C7492AC87245E1
:1051C0008C43EF20A00497B701009387A74848CCF1
:1051D00072458C434249EF206003CA85EF10C06AD4
:1051E00097B70100938707472AC872458C43EF2081
:1051F000E00197B701009387E74508D08C437245DB
:105200004249EF20A000CA85EF10006897B701005F
:10521000938747442AC872458C43EF10307F97B775
:1052200001009387274348D072458C434249EF10D1
:10523000F07DCA85EF1040652AC80840D245EF10BE
:10524000A0642ACA4840D245EF1000642ACA084424
:10525000D245EF1060632ACA4844D245EF10C062BD
:105260002ACA0848D245EF1020622ACA4848D245C7
:10527000EF1080612ACA084CD245EF10E0602ACABC
:10528000484CD245EF1040602ACA0850D245EF1072
:10529000A05F2ACA4850D245EF10005F2ACA424593
:1052A000D245EF20A02D2ACC624593050000EF10D7
:1052B0003069634C050297B701009387A7386245B0
:1052C0008C43EF10305B3325A00009EDA247E39D2E
:1052D00007DE3247835707008507C207C1832310C3
:1052E000F700DDB385473EC4C5B397B70100938788
:1052F000A73662458C43EF10B0647D81F9B71D710C
:105300002AC613058002A2CCA6CACEC6D2C4D6C273
:10531000DAC05EDE62DC66DA6AD86ED686CECAC8CD
:10532000EFE03FB197B701009387473384432A8466
:1053300002C4A68D268DA68C268CA68B268BA68ACB
:10534000268AA689930700003EC83ECA3ECE724513
:10535000A685EF10605308C072454249EE85EF10F4
:10536000A052CA85EF1040522AC87245EA85EF1054
:10537000A05148C072454249E685EF10E050CA8509
:10538000EF1080502AC87245E285EF10E04F08C444
:1053900072454249DE85EF10204FCA85EF10C04E9E
:1053A0002AC87245DA85EF10204E48C4724542493A
:1053B000D685EF10604DCA85EF10004D2AC87245A2
:1053C000D285EF10604C08C872454249CE85EF1077
:1053D000A04BCA85EF10404B97B701009387072871
:1053E0002AC872458C43EF10204A97B70100938773
:1053F000E72648C872458C434249EF10E048CA8509
:10540000EF10804897B70100938747252AC8724557
:105410008C43EF10604797B701009387272408CC8F
:1054200072458C434249EF102046CA85EF10C045B3
:1054300097B70100938787222AC872458C43EF10E3
:10544000A04497B701009387672148CC72458C43ED
:105450004249EF106043CA85EF10004397B701003F
:105460009387C71F2AC872458C43EF10E04197B756
:1054700001009387A71E08D08C4372454249EF1064
:10548000A040CA85EF10404097B701009387071DE1
:105490002AC872458C43EF10203F97B701009387CD
:1054A000E71B48D072458C434249EF10E03DCA8566
:1054B000EF10803D2AC80840D245EF10E03C2ACAD0
:1054C0004840D245EF10403C2ACA0844D245EF106C
:1054D000A03B2ACA4844D245EF10003B2ACA0848DC
:1054E000D245EF10603A2ACA4848D245EF10C03979
:1054F0002ACA084CD245EF1020392ACA484CD24556
:10550000EF1080382ACA0850D245EF10E0372ACA77
:105510004850D245EF1040372ACA4245D245EF20C5
:10552000E0052ACC624593050000EF107041634C02
:10553000050297B701009387E71062458C43EF108F
:1055400070333325A00009EDA247E39D07DE324703
:10555000835707008507C207C1832310F700DDB317
:1055600085473EC4C5B397B701009387E70E6245F0
:105570008C43EF10F03C7D81F9B7411122C42A879A
:105580002A848148014881479746030093868633E1
:105590001306004097B501009385C5EE170500007E
:1055A0001305E59306C6EFB07FCD228781480148F9
:1055B000814797460300938606311306004097B54E
:1055C00001009385A5EC170500001305859EEFB03B
:1055D000FFCA228781480148814797460300938686
:1055E000A62E1306004097B501009385A5EA17057E
:1055F0000000130505D1EFB07FC82287814801481C
:105600008147974603009386462C1306004097B5C2
:1056100001009385A5E8170500001305C5A6EFB0A6
:10562000FFC522878148014881479746030093863A
:10563000E6291306004097B501009385A5E61705F6
:1056400000001305C589EFB07FC322878148014858
:10565000814797460300938686271306004097B537
:1056600001009385A5E41705000013058594EFB0AC
:10567000FFC02287814801488147974603009386EF
:1056800026251306004097B501009385A5E217056E
:105690000000130505C7EFB07FBE22872244B24049
:1056A0008148014881479746030093868622130666
:1056B000004097B50100938565E0170500001305CC
:1056C000859C41016FB09FBB174803000358881F9A
:1056D0001747030003572720174E0300035E8E1E53
:1056E0009746030083D6261E9747030083D7871E5D
:1056F000174303000353231D174503000355C51D1E
:10570000174603000356461C158F9748030083D89D
:10571000A81B9745030083D5451C9746030083D6F5
:10572000C61AB3870741118D3337E00017480300CD
:105730000358A819174603000356461A974F03004B
:1057400083DFCF183307E040958DB337F000333552
:10575000A000974E030083DE6E179746030083D6A2
:105760000618174F0300035F8F16F98F3305A0400B
:105770003306F641B335B000974F030083DF2F1592
:10578000174703000357C7159743030083D34314F8
:10579000E98FB305B040B386E6413336C000174FFA
:1057A0000300035FEF12174503000355851397426B
:1057B000030083D20212ED8F3306C04033077740D7
:1057C000B336D000B306D040F18F330555403337A0
:1057D000E000F58F3307E0403335A000F98F330543
:1057E000A040174703000357C70E974603002393B3
:1057F000C60F974603002390660E97460300239D2D
:10580000160D97460300239A060D9746030023972B
:10581000D60D974603002394F60D97460300239177
:10582000E60D97460300239EE60A7D8D82800000E8
:10583000B305B500930705006386B70003C70700EB
:10584000631607003385A740678000009387170021
:105850006FF09FFE130101FB23229104232C4103CF
:1058600023229103232611042324810423202105CC
:10587000232E3103232A5103232861032326710396
:10588000232481032320A103232EB101930C0500BF
:10589000138A05009304000063DE05003305A04071
:1058A0003337A000B305B040930C0500338AE540C0
:1058B0009304F0FF63DA06003306C040B337C0003C
:1058C000B306D040B386F640930A060093890600DB
:1058D00013840C0013090A006396062817BB010005
:1058E000130BCBA46370CA16B70701006372F614DA
:1058F0009307F00F63F4C70093098000B357360194
:10590000330BFB0083470B0013050002B3873701FD
:10591000B309F540638C0900B3153A01B3D7FC0015
:10592000B31A360133E9B70033943C0113DB0A01A3
:1059300093050B0013050900EF200013130A05005F
:1059400093050B00939B0A0113050900EF20400DFE
:1059500093DB0B019305050013850B00EF208009F5
:10596000131A0A0193570401B367FA0063FAA700F8
:10597000B387570163E6570163F4A700B387570164
:105980003389A74093050B0013050900EF20C00DD4
:10599000130A050093050B0013050900EF204008CA
:1059A0001314040193050500131A0A0113850B0053
:1059B00013540401EF20000433648A00637AA400C6
:1059C00033045401636654016374A4003304540126
:1059D0003304A4403354340193050000638A040067
:1059E00033048040B3378000B305B040B385F54041
:1059F000130504008320C10403248104832441048B
:105A0000032901048329C103032A8103832A410353
:105A1000032B0103832BC102032C8102832C41023F
:105A2000032D0102832DC1011301010567800000D0
:105A3000B707000193090001E362F6EC93098001C6
:105A40006FF0DFEB631A06009305000013051000EA
:105A5000EF10107D930A0500B707010063FAFA0EF4
:105A60009307F00F63F4570193098000B3D73A010D
:105A7000330BFB0083470B001305000233095A4127
:105A8000B3873701B309F540E38209EAB39A3A01D3
:105A9000335BFA00B3153A01B3D7FC0093DB0A017C
:105AA00033E9B70013050B0093850B00EF10D07B93
:105AB000130A050093850B00139C0A0113050B00C4
:105AC000EF101076135C0C019305050013050C0014
:105AD000EF105072131A0A0193570901B367FA00C5
:105AE00033943C0163FAA700B387570163E657017B
:105AF00063F4A700B3875701338BA74093850B004E
:105B000013050B00EF105076130A050093850B0068
:105B100013050B00EF10D0709305050013050C0062
:105B2000EF10506D93160901131A0A0193D606015E
:105B3000B366DA0063FAA600B386560163E656013F
:105B400063F4A600B38656013389A6406FF01FDECA
:105B5000B707000193090001E3EAFAF09309800115
:105B60006FF0DFF06376DA0093050A006FF01FE74D
:105B7000B707010063FAF604930BF00F33B5DB00AF
:105B80001315350033D7A60097A701009387077A2E
:105B9000B387E70083CB070093050002B38BAB000C
:105BA000338B7541631C0B0263E4460163EACC004E
:105BB0003384CC40B306DA4033B98C0033892641B4
:105BC000930509006FF09FE1B7070001130500017D
:105BD000E3EAF6FA130580016FF0DFFAB396660187
:105BE000335D7601336DDD00B35D7A01B3156A0173
:105BF00033DC7C0113540D01336CBC0013850D00A4
:105C000093050400B3196601EF101066930A0500AE
:105C10009305040013850D0033996C01931C0D014D
:105C2000EF10106093DC0C01130A050093050500CA
:105C300013850C00EF10105C939A0A0113570C01A6
:105C400033E7EA00930D0A00637EA7003307A7013C
:105C5000930DFAFF6368A7016376A700930DEAFF2F
:105C60003307A701330AA7409305040013050A0070
:105C7000EF10905F93050400930A050013050A00D6
:105C8000EF10105A930505001304050013850C004E
:105C9000EF10505693150C01939A0A0193D5050104
:105CA000B3E5BA001307040063FEA500B385A501A0
:105CB0001307F4FF63E8A50163F6A5001307E4FFEB
:105CC000B385A501939D0D01B70C0100B3EDED0067
:105CD0001384FCFFB3F78D0033F48900338AA540A9
:105CE00013850700930504002326F10093DD0D01C1
:105CF000EF10505093050400930A050013850D0022
:105D0000EF10504F13DC090193050C002324A10070
:105D100013850D00EF10104E8327C10013040C00F3
:105D200093050400130C050013850700EF10904C39
:105D30008326810013D70A013305D5003307A70056
:105D40006374D700330C9C01B70701009387F7FFFA
:105D5000935507013377F70013170701B3F7FA00DC
:105D6000B3858501B307F7006366BA00631EBA0006
:105D7000637CF90033863741B3B7C700B385A541CB
:105D8000B385F54093070600B307F9403339F900AE
:105D9000B305BA40B385254133947501B3D7670184
:105DA0003364F400B3D565016FF05FC3130101FDE7
:105DB00023229102232A5101232611022324810246
:105DC00023202103232E3101232C410123286101AB
:105DD0002326710123248101232291012320A10183
:105DE000930A050093840500639E06381304060099
:105DF0009309050017A901001309495363F8C51257
:105E0000B7070100138B05006378F6101307F00F36
:105E10003337C70013173700B357E6003309F900CB
:105E2000834609003387E60093060002B386E64006
:105E3000638C0600B394D40033D7EA003314D60041
:105E4000336B9700B399DA00935A040193850A00E3
:105E500013050B00EF1050411309050093850A004C
:105E6000931B040113050B00EF10903B93DB0B0118
:105E7000930405009305050013850B00EF10903780
:105E80001319090193D70901B367F900138A0400B4
:105E900063FEA700B3878700138AF4FF63E88700D7
:105EA00063F6A700138AE4FFB3878700B384A74093
:105EB00093850A0013850400EF10103B13090500B9
:105EC00093850A0013850400EF109035939909011A
:105ED00093040500930505001319090113850B00B0
:105EE00093D90901EF101031B36939011386040009
:105EF00063FCA900B30934011386F4FF63E689004B
:105F000063F4A9001386E4FF13140A013364C40088
:105F1000130A00006F000013B70700011307000108
:105F2000E36CF6EE130780016FF01FEF138A060093
:105F3000631A06009305000013051000EF10502EA1
:105F400013040500B7070100637EF4129307F00FF6
:105F500063F48700130A8000B35744013309F90042
:105F6000034709009306000233074701B386E64062
:105F700063940612B3848440130A1000135B040177
:105F800093050B0013850400EF10102E1309050074
:105F900093050B0013850400931B0401EF10502898
:105FA00093DB0B01930405009305050013850B009B
:105FB000EF1050241319090193D70901B367F900B1
:105FC000938A040063FEA700B3878700938AF4FFD7
:105FD00063E8870063F6A700938AE4FFB38787002E
:105FE000B384A74093050B0013850400EF10D0275E
:105FF0001309050093050B0013850400EF105022D0
:1060000093990901930405009305050013190901EB
:1060100013850B0093D90901EF10D01DB369390125
:106020001386040063FCA900B30934011386F4FF4E
:1060300063E6890063F4A9001386E4FF13940A0160
:106040003364C4001305040093050A008320C102D1
:106050000324810283244102032901028329C1010F
:10606000032A8101832A4101032B0101832BC100F3
:10607000032C8100832C4100032D01001301010337
:1060800067800000B7070001130A0001E366F4EC23
:10609000130A80016FF05FEC3314D40033DAE400AC
:1060A000B399DA0033D7EA00935A0401B394D400C9
:1060B00093850A0013050A00336B9700EF10D01A7E
:1060C0001309050093850A0013050A00931B0401B8
:1060D000EF10101593DB0B019304050093050500E9
:1060E00013850B00EF1010111319090113570B0141
:1060F0003367E900138A0400637EA7003307870033
:10610000138AF4FF636887006376A700138AE4FFAD
:1061100033078700B304A74093850A001385040062
:10612000EF1090141309050093850A0013850400ED
:10613000EF10100F930405009305050013850B0065
:10614000EF10500B13170B01135707011319090117
:10615000B367E9001387040063FEA700B3878700D5
:106160001387F4FF63E8870063F6A7001387E4FF53
:10617000B3878700131A0A01B384A740336AEA0081
:106180006FF0DFDF63ECD51EB707010063F4F604A0
:106190001307F00FB335D7009395350033D7B6000A
:1061A00097A7010093878718B387E70003C7070005
:1061B000130A00023307B700330AEA4063160A02E3
:1061C00013041000E3E096E833B6CA001344160047
:1061D0006FF05FE7B707000193050001E3E0F6FC0D
:1061E000930580016FF09FFBB35CE600B396460118
:1061F000B3ECDC0033D4E40093DB0C01B39744012F
:1062000033D7EA0093850B0013050400336BF700C6
:10621000B3194601EF1050051309050093850B00D3
:1062200013050400139C0C01EF10807F135C0C011C
:10623000930405009305050013050C00EF10807B07
:106240001319090113570B013367E9001384040084
:10625000637EA700330797011384F4FF63689701F7
:106260006376A7001384E4FF33079701B304A740C4
:1062700093850B0013850400EF10007F13090500C0
:1062800093850B0013850400EF10807993040500BB
:106290009305050013050C00EF10C07593170B0153
:1062A0001319090193D70701B367F9001386040096
:1062B00063FEA700B38797011386F4FF63E8970195
:1062C00063F6A7001386E4FFB38797011314040154
:1062D000B70B01003364C4001389FBFF337D240135
:1062E00033F92901B384A7409305090013050D0074
:1062F000EF104070935C040193050900130B050037
:1063000013850C00EF10006F93D90901130C0500E1
:106310009385090013850C00EF10C06D130905006B
:106320009385090013050D00EF10C06C330585013E
:1063300093570B013385A7006374850133097901F5
:1063400093570501B387270163E6F402E392F4BC97
:10635000B70701009387F7FF3375F50013150501A3
:10636000337BFB0033964A0133056501130A0000B5
:10637000E37AA6CC1304F4FF6FF09FB9130A000070
:10638000130400006FF01FCC130101FB23248104D0
:1063900023229104232E3103232291032326110467
:1063A00023202105232C4103232A510323286103A1
:1063B00023267103232481032320A103232EB1016B
:1063C000930C0500938905001304050093840500D0
:1063D000639E062613090600138A060097AA010089
:1063E000938ACAF463F4C514B70701006376F61202
:1063F0009307F00F63F4C700130A8000B3574601F8
:10640000B38AFA0003C70A001305000233074701E5
:10641000330AE540630C0A00B395490133D7EC0019
:1064200033194601B364B70033944C01935A090100
:1064300093850A0013850400EF100063930905009B
:1064400093850A00131B090113850400EF10405DBA
:10645000135B0B019305050013050B00EF1080592A
:106460009399090193570401B3E7F90063FAA70070
:10647000B387270163E6270163F4A700B3872701E9
:10648000B384A74093850A0013850400EF10C05D14
:106490009309050093850A0013850400EF10405806
:1064A00013140401930505009399090113050B00CA
:1064B00013540401EF10005433E48900637AA400FC
:1064C00033042401636624016374A40033042401AB
:1064D0003304A44033554401930500008320C104D4
:1064E0000324810483244104032901048329C10373
:1064F000032A8103832A4103032B0103832BC10257
:10650000032C8102832C4102032D0102832DC10142
:106510001301010567800000B7070001130A00019D
:10652000E36EF6EC130A80016FF05FED631A06006C
:106530009305000013051000EF10804E13090500AD
:10654000B7070100637AF90E9307F00F63F4270190
:10655000130A8000B3574901B38AFA0003C70A003F
:1065600013050002B384294133074701330AE5408C
:10657000E30E0AEA33194901B3DAE900B395490198
:1065800033D7EC0093540901336BB70013850A002D
:1065900093850400EF10404D930905009385040096
:1065A000931B090113850A00EF10804793DB0B0151
:1065B0009305050013850B00EF10C0439399090163
:1065C00093570B01B3E7F90033944C0163FAA7002A
:1065D000B387270163E6270163F4A700B387270188
:1065E000B38AA7409385040013850A00EF10C047C3
:1065F000930905009385040013850A00EF104042BB
:106600009305050013850B00EF10C03E93150B0199
:106610009399090193D50501B3E5B90063FAA50083
:10662000B385250163E6250163F4A500B385250143
:10663000B384A5406FF09FDFB7070001130A000184
:10664000E36AF9F0130A80016FF0DFF0E3E8D5E8C0
:10665000B707010063FCF604930BF00F33B5DB00C2
:106660001315350033D7A60097A70100938707CCF1
:10667000B387E70083CB070093050002B38BAB0021
:10668000338B7541631E0B0263E4360163EACC0071
:106690003384CC40B386D94033B58C00B384A64054
:1066A00013050400938504006FF05FE3B707000152
:1066B00013050001E3E8F6FA130580016FF09FFA75
:1066C000B3966601335D7601336DDD0033D4790115
:1066D000B395690133DC7C0193540D01336CBC002C
:1066E0001305040093850400B31A6601EF10C03748
:1066F000130A0500938504001305040033996C0107
:10670000931C0D01EF10C03193DC0C011304050044
:106710009305050013850C00EF10C02D131A0A0114
:1067200013570C013367EA00130A0400637EA700C5
:106730003307A701130AF4FF6368A7016376A70074
:10674000130AE4FF3307A701B309A74093850400A8
:1067500013850900EF1040319385040013040500F0
:1067600013850900EF10C02B930505009304050065
:1067700013850C00EF10002893150C01131404016D
:1067800093D50501B365B4001387040063FEA5002B
:10679000B385A5011387F4FF63E8A50163F6A5009F
:1067A0001387E4FFB385A501131A0A01B70C010092
:1067B000336AEA001384FCFFB3778A0033F48A005B
:1067C000B384A54013850700930504002326F10038
:1067D000135A0A01EF1000229309050093050400E3
:1067E00013050A00EF10002113DC0A01930D0500C8
:1067F00093050C0013050A00EF10C01F8327C1008A
:10680000130A050093050C0013850700EF10801E86
:106810003305B50113D709013307A7006374B70126
:10682000330A9A01B70701009387F7FF93550701D1
:106830003377F70013170701B3F7F900B385450164
:10684000B307F70063E6B400639EB400637CF9000D
:1068500033865741B3B7C700B385A541B385F5402B
:1068600093070600B307F9403339F900B385B44004
:10687000B385254133947501B3D767013365F400BF
:10688000B3D565016FF09FC5B7078000130101FF05
:106890009387F7FF33F7A7002324810023202101EA
:1068A000135475011359F50113D57501B3F7B700EA
:1068B0001374F40F1375F50F232611002322910092
:1068C00093D5F50113163700939737003307A4408B
:1068D000631EB9186358E00A63180506639C070035
:1068E0009307F00F630CF4049307060013050400EC
:1068F0006F00C00B1307F7FF631E0702B387C700C3
:1069000013050400139757006352070A1305150077
:106910001307F00F6304E5323707007E93F6170084
:106920001307F7FF93D71700B3F7E700B3E7D700D4
:106930006F00C0079306F00F6310D40293070600A0
:106940001305F00F6F0080069306F00FE308D4FEE6
:10695000B7060004B3E7D7009306B00163D6E6009C
:10696000930710006FF09FF993060002B386E6408C
:10697000B3D5E700B397D700B337F000B3E7F5001E
:106980006FF0DFF763040708631004046300060276
:106990009306F0FF6316D700B387C7006FF09FF62A
:1069A0009306F00F1347F7FF631AD50213F777002A
:1069B0006308072813F7F700930640006302D728FF
:1069C000938747006F00C0279306F00FE300D5FEC2
:1069D000B70600043307E0403366D6009306B001E3
:1069E00063D6E600130710006F00C0019306000293
:1069F000B355E6003387E6403317E6003337E0004F
:106A000033E7E500B387E7006FF0DFEF130514000D
:106A10009376F50F130710006340D7046318040240
:106A200013050000E30406F863860720B387C70058
:106A300013975700E35C07F6370700FC1307F7FFCF
:106A4000B3F7E700130510006FF05FF6E30A06EEF8
:106A5000639407166FF09FEE1307F00F6300E51EB7
:106A60003307F600935717006FF05FF46350E008A8
:106A700063160504E38607E61307F7FF63140702AE
:106A8000B307F6401305040013975700E35007F2CD
:106A9000B70400049384F4FFB3F4970013040500D3
:106AA0006F00C0139306F00FE30AD4E89306B00119
:106AB00063D0E602930710006FF09FFC9306F00F7F
:106AC000E30ED4E6B7060004B3E7D7006FF01FFE6D
:106AD00093060002B3D5E7003387E640B397E7009B
:106AE000B337F000B3E7F5006FF09FF9630E0706C8
:106AF000631E040213890500E30A06EA9306F0FF09
:106B00006318D700B387C740138905006FF0DFF71C
:106B10009306F00F1347F7FFE30AD5E89306B00199
:106B200063D4E602130710006F0080039306F00F92
:106B300013890500E30CD5E6B70600043307E040EF
:106B40003366D6006FF09FFD930600023358E600CF
:106B50003387E6403317E6003337E0003367E80059
:106B6000B387E7406FF05FFA130714001377F70F4E
:106B70009306100063CAE604631C0402631806004F
:106B8000639E0712130500006F008003638C0712D9
:106B90003307F64093165700B387C74063C0061209
:106BA0009307070063160706930700006FF09FFD29
:106BB000E31006EA639C0710B70700021305F00F05
:106BC000130900006F00C007B304F6401397540088
:106BD00063540704B384C740138905001385040078
:106BE000EF00D06E1305B5FFB394A400634A85028D
:106BF000330585401305150013040002B3D7A40024
:106C00003305A440B394A400B3349000B3E79700D5
:106C1000130500006FF09FD9E38804F86FF01FFCA4
:106C2000B70700FC9387F7FF3305A440B3F7F400E0
:106C30006FF0DFD7930706006FF05FD79307000070
:106C400013975700635E0700130515001307F00F35
:106C50006302E508370700FC1307F7FFB3F7E70007
:106C60001307F00F93D737006318E500638607001A
:106C7000B707400013090000370780001307F7FF2C
:106C80001375F50FB3F7E70013177501370580800B
:106C90008320C100032481001305F5FF33F5A7000D
:106CA0001319F9013365E50033652501832441009B
:106CB0000329010013010101678000001389050009
:106CC0006FF01FF5930706006FF09FF4138905001E
:106CD0006FF01FC7930700006FF09FF8130101FDCD
:106CE00023229102232A510193547501B70A80008F
:106CF0002320210323286101938AFAFF232611020E
:106D000023248102232E3101232C410123267101EA
:106D10002324810193F4F40F138B0500B3FAAA0026
:106D20001359F501638804089307F00F6384F40A8C
:106D3000939A3A00B7070004B3EAFA00938414F870
:106D4000930B000013557B01370480001304F4FFFC
:106D50001375F50F33746401135BFB01630C0508B5
:106D60009307F00F6308F50A13143400B707000403
:106D70003364F400130515F89307000013972B00F4
:106D80003367F7001307F7FF9306E000B349690183
:106D9000338AA44063E0E60A979601009386865101
:106DA000131727003307D700032707003307D7003F
:106DB00067000700638A0A0213850A00EF0010517A
:106DC0009307B5FF9304A0F8B39AFA00B384A440E4
:106DD0006FF01FF79304F00F930B2000E3840AF683
:106DE000930B30006FF01FF693040000930B10001C
:106DF0006FF05FF5630A040213050400EF00104D05
:106E00009307B5FF3314F4009307A0F83385A74028
:106E10006FF09FF61305F00F93072000E30004F6D0
:106E2000930730006FF09FF51305000093071000E3
:106E30006FF0DFF4131B540063F68A12130AFAFF93
:106E400013090000935B0B013704010093850B00CD
:106E50001304F4FF13850A00EF00903C33748B0099
:106E600093050500130C050013050400EF0090388E
:106E70009304050093850B0013850A00EF00D03EB4
:106E800013590901131505013365A90013090C00F5
:106E9000637E9500330565011309FCFF6368650196
:106EA000637695001309ECFF33056501B304954043
:106EB00093850B0013850400EF00903693050500C1
:106EC000130C050013050400EF00D032930A0500EF
:106ED00093850B0013850400EF001039131505018D
:106EE00013040C00637E5501330565011304FCFF98
:106EF00063686501637655011304ECFF3305650192
:106F00001319090133055541336989003335A00050
:106F10003364A9001307FA076350E00A93777400FB
:106F2000638A07009377F400930640006384D700D8
:106F3000130444009317440063DA0700B70700F80E
:106F40009387F7FF3374F40013070A089307E00FE1
:106F50001354340063D2E70C130400001307F00F3E
:106F60006F00800B1399FA0193DA1A006FF09FED0E
:106F70009309090013840A0093870B00130720006C
:106F8000E38CE7FC130730006382E7081307100067
:106F9000E392E7F813040000130700006F00C00736
:106FA00093090B006FF09FFD370440009309000028
:106FB000930730006FF09FFC93071000B387E74002
:106FC0001307B001E348F7FC1305EA09B357F400CF
:106FD0003314A4003334800033E4870093777400C3
:106FE000638A07009377F400130740006384E70087
:106FF000130444009317540013543400E3DE07F8DD
:1070000013040000130710006F0000013704400054
:107010001307F00F93090000370580001305F5FFF3
:107020003374A400370580801305F5FF1377F70F3D
:107030003374A400131777011395F9013364E40046
:107040003365A4008320C10203248102832441020A
:10705000032901028329C101032A8101832A4101F5
:10706000032B0101832BC100032C810013010103B9
:1070700067800000370780001307F7FF93567501FC
:107080003378A70013D675019357F50193F6F60FE1
:107090001305F00F3377B7001376F60F93D5F5018C
:1070A0006398A6001305E0FF630E080667800000E2
:1070B0006318A6001305E0FF630E07066780000053
:1070C000639406061335180063140600630607046C
:1070D000631C05006394B700635ED60013051000BF
:1070E0006396070067800000E39E05FE1305F0FF2E
:1070F0006780000063DAC6001305F0FFE38407FE33
:107100001305100067800000E36A07FD1305000007
:10711000E364E8FE6FF01FFD13050000E30408FCC4
:107120006FF0DFFBE308D6F8E31606FAE30807FA88
:107130006FF05FFA13351800E38C06F86FF09FF9D3
:10714000370780001307F7FF935675013378A700C0
:1071500013D675019357F50193F6F60F1305F00F4B
:107160003377B7001376F60F93D5F5016398A60031
:1071700013052000630E0806678000006318A60050
:1071800013052000630E070667800000639406065F
:10719000133518006314060063060704631C05001A
:1071A0006394B700635ED600130510006396070072
:1071B00067800000E39E05FE1305F0FF6780000076
:1071C00063DAC6001305F0FFE38407FE1305100021
:1071D00067800000E36A07FD13050000E364E8FE32
:1071E0006FF01FFD13050000E30408FC6FF0DFFBE8
:1071F000E308D6F8E31606FAE30807FA6FF05FFA39
:1072000013351800E38C06F86FF09FF9130101FDA8
:107210002322910223202103B70480001359750112
:10722000232E3101232671019384F4FF23261102BA
:1072300023248102232C4101232A510123286101A7
:1072400023248101232291011379F90F938B0500E7
:10725000B3F4A4009359F501630A09089307F00FEA
:107260006306F90A93943400B7070004B3E4F4000A
:10727000130919F8130B000013D57B0137048000A4
:107280001304F4FF1375F50F3374740193DBFB01E2
:10729000630E05089307F00F630AF50A1314340010
:1072A000B70700043364F400130515F893060000D3
:1072B00093172B00B3E7D7003309A9009387F7FF93
:1072C0001307E00033CA7901930A19006360F70AD3
:1072D000179701001307C70193972700B387E700AB
:1072E00083A70700B387E70067800700638A04026B
:1072F00013850400EF00807D9307B5FF1309A0F804
:10730000B394F4003309A9406FF0DFF61309F00FCE
:10731000130B2000E38204F6130B30006FF0DFF54F
:1073200013090000130B10006FF01FF5630A04022D
:1073300013050400EF0080799307B5FF3314F400C0
:107340009307A0F83385A7406FF05FF61305F00FA1
:1073500093062000E30E04F4930630006FF05FF50F
:1073600013050000930610006FF09FF4370C010026
:10737000130BFCFF93DB0401935C0401B3F4640181
:10738000337464019305040013850400EF008066E4
:10739000930504009309050013850B00EF00806539
:1073A0001304050093850C0013850B00EF00806427
:1073B000930B05009385040013850C00EF00806398
:1073C0003305850093D709013385A70063748500D1
:1073D000B38B8B01B377650193970701B3F969010B
:1073E000B3873701139467003334800093D7A70124
:1073F00013550501B367F4003304750113146400D9
:107400003364F4009317440063D6070E93571400B7
:107410001374140033E487001387FA076350E00EF7
:1074200093777400638A07009377F4009306400013
:107430006384D700130444009317440063DA070001
:10744000B70700F89387F7FF3374F40013870A082F
:107450009307E00F63C4E710935734006F000003F5
:10746000138A09001384040093060B00930720007D
:107470006386F60E93073000638AF60C130610003D
:107480009307000013070000E398C6F83704800054
:107490001304F4FF37058080B3F787001305F5FF69
:1074A0008320C102032481021377F70FB3F7A700EB
:1074B000131777011315FA01B3E7E700832441029C
:1074C000032901028329C101032A8101832A410181
:1074D000032B0101832BC100032C8100832C41006D
:1074E00033E5A7001301010367800000138A0B0036
:1074F0006FF0DFF7930A09006FF01FF29307100097
:10750000B387E7401307B0016340F706938AEA099F
:10751000B357F400331454013334800033E487004C
:1075200093777400638A07009377F4001307400091
:107530006384E700130444009317540063CA0702EE
:1075400093573400130700006FF05FF4B707400053
:107550001307F00F130A00006FF05FF393070000AA
:107560001307F00F6FF09FF2930700006FF09FFD7D
:1075700093070000130710006FF05FF1B70780005A
:107580009387F7FF130101FF33F7A70093567501A7
:1075900013D67501B3F7B7002322910023202101F0
:1075A00093F6F60F131837001376F60F2326110003
:1075B000232481001307F00F9354F501138906006B
:1075C0001305060093D5F501939737006314E60081
:1075D0006394070093C515003387C640639A951AD4
:1075E0006356E00A63160606639C07009307F00FD4
:1075F000638CF60493070800138506006F00C0141F
:107600001307F7FF631E0702B38707011385060000
:1076100013975700635A0712130515001307F00F4D
:10762000630EE5323707007E93F617001307F7FF66
:1076300093D71700B3F7E700B3E7D7006F00C01088
:107640001306F00F639EC600930708006F00400703
:107650001306F00FE38AC6FE37060004B3E7C7003F
:107660001306B0016356E600930710006FF0DFF9D0
:10767000130600023306E640B3D5E700B397C70010
:10768000B337F000B3E7F5006FF01FF863000708A9
:10769000639C0602631808001307F00F6316E60ADE
:1076A0006F0000029306F0FF6316D700B38707014F
:1076B0006FF01FF69306F00F1347F7FF6310D60223
:1076C0001305F00F6F0040089306F00FE30AD6FE93
:1076D000B70600043307E0403368D8009306B001D2
:1076E00063D6E600130710006F00C0019306000286
:1076F0003356E8003387E6403317E8003337E000BD
:107700003367E600B387E7006FF09FF0138516003C
:107710001376F50F130710006342C706639406043F
:10772000130500006302080263860722B38707017E
:1077300013975700635A0700370700FC1307F7FF3A
:10774000B3F7E7001305100013F77700630A07206B
:1077500013F7F700930640006304D7209387470090
:107760006F000020E30E08F4E38007EEB707000285
:107770001305F00F930400006F00801E1307F00F35
:10778000630EE51C3307F800935717006FF0DFFB1B
:107790006350E00863160604E38A07E41307F7FF63
:1077A00063140702B307F8401385060013975700C8
:1077B000E35C07F8370400041304F4FF33F4870094
:1077C000130905006F0080131306F00FE38EC6E661
:1077D0001306B0016350E602930710006FF09FFCA0
:1077E0001306F00FE382C6E637060004B3E7C700CE
:1077F0006FF01FFE13060002B3D5E7003307E64023
:10780000B397E700B337F000B3E7F5006FF09FF9E7
:1078100063020708639E0602631808001307F00F4F
:10782000938405006FF09FE79306F0FF6318D7007D
:10783000B3870741938405006FF05FF79306F00F5D
:107840001347F7FF6310D602938405006FF05FE7DC
:107850009306F00FE30AD6FEB70600043307E040B4
:107860003368D8009306B00163D6E6001307100012
:107870006F00C001930600023356E8003387E640EC
:107880003317E8003337E0003367E600B387E7409B
:107890006FF05FFA138716001377F70F13061000C7
:1078A0006344E604639C06026318080063980712A9
:1078B000130500006FF01FEC638607123307F840D2
:1078C00093165700B387074163CA06109307070052
:1078D00063100706930700006FF09FFDE31608E8AA
:1078E000E39407F66FF09FE83304F8401317540051
:1078F000635407043384074193840500130504008F
:10790000EF00C01C1305B5FF3314A400634A250320
:10791000330525411305150013070002B357A400D2
:107920003305A7403314A40033348000B3E7870045
:10793000130500006FF05FE1E30E04F86FF01FFC29
:10794000B70700FC9387F7FF3305A940B377F4002E
:107950006FF09FDF930708006FF01FDF93070000B1
:1079600013975700635E0700130515001307F00F08
:10797000630EE506370700FC1307F7FFB3F7E700D0
:107980001307F00F93D737006318E50063860700ED
:10799000B707400093040000370780001307F7FF84
:1079A0001375F50FB3F7E7001317750137058080DE
:1079B0008320C100032481001305F5FF33F5A700E0
:1079C0009394F4013365E5003365950003290100C4
:1079D00083244100130101016780000093840500A6
:1079E0006FF01FF5930708006FF09FF493070000F6
:1079F0006FF01FF9130605001305000093F615003C
:107A0000638406003305C50093D5150013161600D0
:107A1000E39605FE678000006340050663C6050621
:107A200013860500930505001305F0FF630C06029D
:107A300093061000637AB6006358C0001316160050
:107A400093961600E36AB6FE1305000063E6C500D0
:107A5000B385C5403365D50093D61600135616007E
:107A6000E39606FE6780000093820000EFF05FFB64
:107A700013850500678002003305A04063D8050028
:107A8000B305B0406FF0DFF9B305B040938200005A
:107A9000EFF01FF93305A0406780020093820000D9
:107AA00063CA0500634C0500EFF09FF713850500DE
:107AB00067800200B305B040E35805FE3305A040DF
:107AC000EFF01FF63305B04067800200B7070100F2
:107AD000637AF5029307F00FB3B7A70093973700C7
:107AE000130700023307F740B357F500179501005D
:107AF0001305C583B307F50003C507003305A74089
:107B0000678000003707000193070001E36AE5FC86
:107B1000930780016FF0DFFC97970100938787AE92
:107B20009443179701001307A7AC1843C8C2637B9F
:107B3000E50017970100130767AC08438C439105D4
:107B40006F801FA0411122C406C6179701001307BA
:107B500027AB2A8408438C439105EF807F9E97973B
:107B60000100938727A79C436376F4009797010051
:107B700023A287A6B2402244410182809797010048
:107B8000938747A8984394437C43FD177CC3FC42EA
:107B900099E3736004308280011122CC26CA2A84C2
:107BA000AE844AC84EC652C456C206CEEFA02F9627
:107BB0001C4003290401B7090001B3E59700930AAB
:107BC000C4000CC08144FD19370A00021840638CC0
:107BD0002A03032609004A85B3654701B3763601B7
:107BE00093175600758F0329490063C4070001E706
:107BF000F1BFE39DE6FC9317760063D30700D58CB5
:107C0000EFB04F80E1B793C4F4FFF98C04C0EFA04C
:107C10000FB50840F2406244D2444249B249224A78
:107C2000924A056182804111014506C622C4EFD007
:107C3000DF9417D7FFFF1307071A81460546930500
:107C400040061795010013052583EFB0BFCF19C972
:107C50002A84EFA0CF8C2A8601478146854522855C
:107C6000EFB0FFDAEF903FE5B24022440145410119
:027C7000828010
:02000004800278
:10000000CE44FEFFCC45FEFFD644FEFFCC45FEFFAE
:10001000CC45FEFFCC45FEFFCC45FEFFEE44FEFF87
:10002000CC45FEFFCC45FEFF0845FEFF1445FEFF14
:10003000CC45FEFF2645FEFF3245FEFF3245FEFF62
:100040003245FEFF3245FEFF3245FEFF3245FEFFE0
:100050003245FEFF3245FEFF3245FEFFCC45FEFF36
:10006000CC45FEFFCC45FEFFCC45FEFFCC45FEFF58
:10007000CC45FEFFCC45FEFFCC45FEFFCC45FEFF48
:10008000CC45FEFFCC45FEFFCC45FEFFCC45FEFF38
:10009000CC45FEFFCC45FEFFCC45FEFFCC45FEFF28
:1000A000CC45FEFFCC45FEFFCC45FEFFCC45FEFF18
:1000B000CC45FEFFCC45FEFFCC45FEFFCC45FEFF08
:1000C000CC45FEFFCC45FEFFCC45FEFFCC45FEFFF8
:1000D000CC45FEFFCC45FEFFCC45FEFFCC45FEFFE8
:1000E000CC45FEFFCC45FEFFCC45FEFFCC45FEFFD8
:1000F000CC45FEFFCC45FEFFCC45FEFFCC45FEFFC8
:100100006645FEFF7C45FEFFCC45FEFFCC45FEFF6D
:10011000CC45FEFFCC45FEFFCC45FEFFCC45FEFFA7
:10012000CC45FEFFC245FEFFCC45FEFFCC45FEFFA1
:100130007443FEFF2C44FEFFCC45FEFFCC45FEFF82
:100140006244FEFFCC45FEFFBA44FEFFCC45FEFFF5
:10015000CC45FEFFE844FEFFDA48FEFF2E49FEFFD5
:10016000E248FEFF2E49FEFF2E49FEFF2E49FEFF0C
:100170002E49FEFFD447FEFF2E49FEFF2E49FEFF0B
:10018000EE47FEFFFA47FEFF2E49FEFF0C48FEFF3A
:100190001848FEFF1848FEFF1848FEFF1848FEFFEB
:1001A0001848FEFF1848FEFF1848FEFF1848FEFFDB
:1001B0001848FEFF2E49FEFF2E49FEFF2E49FEFF86
:1001C0002E49FEFF2E49FEFF2E49FEFF2E49FEFF5F
:1001D0002E49FEFF2E49FEFF2E49FEFF2E49FEFF4F
:1001E0002E49FEFF2E49FEFF2E49FEFF2E49FEFF3F
:1001F0002E49FEFF2E49FEFF2E49FEFF2E49FEFF2F
:100200002E49FEFF2E49FEFF2E49FEFF2E49FEFF1E
:100210002E49FEFF2E49FEFF2E49FEFF2E49FEFF0E
:100220002E49FEFF2E49FEFF2E49FEFF2E49FEFFFE
:100230002E49FEFF2E49FEFF2E49FEFF2E49FEFFEE
:100240002E49FEFF2E49FEFF2E49FEFF2E49FEFFDE
:100250002E49FEFF2E49FEFF4C48FEFF7A48FEFF66
:100260002E49FEFF2E49FEFF2E49FEFF2E49FEFFBE
:100270002E49FEFF2E49FEFF2E49FEFFD048FEFF0D
:100280002E49FEFF2E49FEFF3246FEFF2C47FEFFA1
:100290002E49FEFF2E49FEFF9E47FEFF2E49FEFF20
:1002A000C447FEFF2E49FEFF2E49FEFF2849FEFFF0
:1002B000A86CFEFFE46CFEFFF06CFEFFE46CFEFF3A
:1002C0005C6DFEFFE46CFEFFF06CFEFFA86CFEFFB1
:1002D000A86CFEFF5C6DFEFFF06CFEFFC06CFEFFC5
:1002E000C06CFEFFC06CFEFFF86CFEFF8071FEFF6D
:1002F0008071FEFF0072FEFF7871FEFF7871FEFFD5
:100300006072FEFF0072FEFF7871FEFF6072FEFFFA
:100310007871FEFF0072FEFF7471FEFF7471FEFFC4
:100320007471FEFF6072FEFF00010202030303030B
:100330000404040404040404050505050505050575
:100340000505050505050505060606060606060655
:10035000060606060606060606060606060606063D
:100360000606060606060606070707070707070725
:10037000070707070707070707070707070707070D
:1003800007070707070707070707070707070707FD
:1003900007070707070707070707070707070707ED
:1003A00007070707070707070808080808080808D5
:1003B00008080808080808080808080808080808BD
:1003C00008080808080808080808080808080808AD
:1003D000080808080808080808080808080808089D
:1003E000080808080808080808080808080808088D
:1003F000080808080808080808080808080808087D
:10040000080808080808080808080808080808086C
:10041000080808080808080808080808080808085C
:100420000808080808080808546D72510000000008
:10043000546D722053766300286E756C6C29000031
:100440004572726F7220696E2073705F666C6F7098
:1004500073207461736B73200D0A00006D69616F06
:10046000750A00006D69616F75320A0068756E6704
:1004700072790A00436865636B54696D65720000A8
:100480004D617468310000004D61746832000000F5
:100490004D617468330000004D61746834000000E1
:1004A0004D617468350000004D61746836000000CD
:1004B0004D617468370000004D61746838000000B9
:1004C0001000000000000000017A5200017C0101D0
:1004D0001B0D020050000000180000007853FEFFC2
:1004E0005805000000440E507489039406990B814E
:1004F00001880292049305950796089709980A9A2D
:100500000C9B0D036C010AC144C844C944D244D3B6
:1005100044D444D544D644D744D844D944DA44DBFF
:10052000440E00440B0000004C0000006C00000072
:100530007C58FEFFDC05000000440E3070890395F6
:1005400007810188029204930594069608970998FA
:100550000A990B9A0C0370020AC144C844C944D2D8
:1005600044D344D444D544D644D744D844D944DAB7
:10057000440E00440B00000050000000BC000000CE
:10058000085EFEFF0005000000440E5074880289DA
:10059000039305990B810192049406950796089799
:1005A00009980A9A0C9B0D0320010AC144C844C94A
:1005B00044D244D344D444D544D644D744D844D96F
:0C05C00044DA44DB440E00440B00000051
:10063400D5E9F642DD9A1245358E65C46F12833AC8
:10064400A4B0C2C366E4FD46A30100C0CFF7414194
:100654006F1283BA0000B040FC8F01000900000053
:040000058000004037
:00000001FF
